 hprof

 Timestamp is 6a16388f (Tue May 26 20:19:27 2026)

 Preferred load address is 10000000

 Start         Length     Name                   Class
 0001:00000000 00017e86H .text$mn                CODE
 0002:00000000 00000164H .idata$5                DATA
 0002:00000164 00000008H .00cfg                  DATA
 0002:0000016c 00000004H .CRT$XCA                DATA
 0002:00000170 00000004H .CRT$XCZ                DATA
 0002:00000174 00000004H .CRT$XIA                DATA
 0002:00000178 00000004H .CRT$XIZ                DATA
 0002:0000017c 00000004H .CRT$XPA                DATA
 0002:00000180 00000004H .CRT$XPZ                DATA
 0002:00000184 00000004H .CRT$XTA                DATA
 0002:00000188 00000008H .CRT$XTZ                DATA
 0002:0000018c 00000000H .gfids$y                DATA
 0002:00000190 000045f0H .rdata                  DATA
 0002:00004780 00000000H .rdata$CastGuardVftablesA DATA
 0002:00004780 00000000H .rdata$CastGuardVftablesC DATA
 0002:00004780 00000004H .rdata$sxdata           DATA
 0002:00004784 000000d0H .rdata$voltmd           DATA
 0002:00004854 000002f4H .rdata$zzzdbg           DATA
 0002:00004b48 00000004H .rtc$IAA                DATA
 0002:00004b4c 00000004H .rtc$IZZ                DATA
 0002:00004b50 00000004H .rtc$TAA                DATA
 0002:00004b54 00000004H .rtc$TZZ                DATA
 0002:00004b58 00000088H .xdata$x                DATA
 0002:00004be0 0000006cH .edata                  DATA
 0002:00004c4c 00000104H .idata$2                DATA
 0002:00004d50 00000014H .idata$3                DATA
 0002:00004d64 00000164H .idata$4                DATA
 0002:00004ec8 0000055cH .idata$6                DATA
 0003:00000000 00000138H .data                   DATA
 0003:00000138 0000070cH .bss                    DATA
 0004:00000000 00000060H .rsrc$01                DATA
 0004:00000060 00000360H .rsrc$02                DATA

  Address         Publics by Value              Rva+Base       Lib:Object

 0000:00000000       ___AbsoluteZero            00000000     <absolute>
 0000:00000000       ___arm64x_extra_rfe_table  00000000     <absolute>
 0000:00000000       ___arm64x_extra_rfe_table_size 00000000     <absolute>
 0000:00000000       ___arm64x_native_entrypoint 00000000     <absolute>
 0000:00000000       ___arm64x_redirection_metadata 00000000     <absolute>
 0000:00000000       ___arm64x_redirection_metadata_count 00000000     <absolute>
 0000:00000000       ___dynamic_value_reloc_table 00000000     <absolute>
 0000:00000000       ___enclave_config          00000000     <absolute>
 0000:00000000       ___guard_check_icall_a64n_fptr 00000000     <absolute>
 0000:00000000       ___guard_eh_cont_count     00000000     <absolute>
 0000:00000000       ___guard_eh_cont_table     00000000     <absolute>
 0000:00000000       ___guard_fids_count        00000000     <absolute>
 0000:00000000       ___guard_fids_table        00000000     <absolute>
 0000:00000000       ___guard_iat_count         00000000     <absolute>
 0000:00000000       ___guard_iat_table         00000000     <absolute>
 0000:00000000       ___guard_longjmp_count     00000000     <absolute>
 0000:00000000       ___guard_longjmp_table     00000000     <absolute>
 0000:00000000       ___hybrid_auxiliary_iat    00000000     <absolute>
 0000:00000000       ___hybrid_auxiliary_iat_copy 00000000     <absolute>
 0000:00000000       ___hybrid_code_map         00000000     <absolute>
 0000:00000000       ___hybrid_code_map_count   00000000     <absolute>
 0000:00000000       ___x64_code_ranges_to_entry_points 00000000     <absolute>
 0000:00000000       ___x64_code_ranges_to_entry_points_count 00000000     <absolute>
 0000:00000001       ___safe_se_handler_count   00000001     <absolute>
 0000:00000100       ___guard_flags             00000100     <absolute>
 0000:00000000       ___ImageBase               10000000     <linker-defined>
 0001:00000000       @_guard_check_icall_nop@4  10001000 f   MSVCRT:guard_support.obj
 0001:00000000       _debug_malloc_police       10001000 f   debug_malloc.obj
 0001:00000000       _io_write_file_footer      10001000 f   hprof_io.obj
 0001:00000000       _io_write_oldprof_footer   10001000 f   hprof_io.obj
 0001:00000000       _io_write_trace_footer     10001000 f   hprof_io.obj
 0001:00000000       _md_init                   10001000 f   hprof_md.obj
 0001:00000010       _blocks_alloc              10001010 f   hprof_blocks.obj
 0001:000000d0       _blocks_init               100010d0 f   hprof_blocks.obj
 0001:00000100       _blocks_term               10001100 f   hprof_blocks.obj
 0001:00000130       _check_binary_file         10001130 f   hprof_check.obj
 0001:00003d00       _class_add_status          10004d00 f   hprof_class.obj
 0001:00003d20       _class_all_status_remove   10004d20 f   hprof_class.obj
 0001:00003d40       _class_cleanup             10004d40 f   hprof_class.obj
 0001:00003d70       _class_create              10004d70 f   hprof_class.obj
 0001:00003da0       _class_delete_global_references 10004da0 f   hprof_class.obj
 0001:00003dc0       _class_do_unloads          10004dc0 f   hprof_class.obj
 0001:00003de0       _class_find_or_create      10004de0 f   hprof_class.obj
 0001:00003e30       _class_get_all_fields      10004e30 f   hprof_class.obj
 0001:00003f10       _class_get_class           10004f10 f   hprof_class.obj
 0001:00004000       _class_get_inst_size       10005000 f   hprof_class.obj
 0001:00004020       _class_get_loader          10005020 f   hprof_class.obj
 0001:00004050       _class_get_methodID        10005050 f   hprof_class.obj
 0001:000042a0       _class_get_object_index    100052a0 f   hprof_class.obj
 0001:000042c0       _class_get_serial_number   100052c0 f   hprof_class.obj
 0001:000042f0       _class_get_signature       100052f0 f   hprof_class.obj
 0001:00004320       _class_get_status          10005320 f   hprof_class.obj
 0001:00004340       _class_get_super           10005340 f   hprof_class.obj
 0001:00004360       _class_init                10005360 f   hprof_class.obj
 0001:00004390       _class_list                10005390 f   hprof_class.obj
 0001:000043c0       _class_new_classref        100053c0 f   hprof_class.obj
 0001:00004450       _class_prime_system_classes 10005450 f   hprof_class.obj
 0001:000044f0       _class_set_inst_size       100054f0 f   hprof_class.obj
 0001:00004510       _class_set_methods         10005510 f   hprof_class.obj
 0001:000045b0       _class_set_object_index    100055b0 f   hprof_class.obj
 0001:000045d0       _class_set_super           100055d0 f   hprof_class.obj
 0001:00004a50       _cpu_sample_init           10005a50 f   hprof_cpu.obj
 0001:00004ad0       _cpu_sample_off            10005ad0 f   hprof_cpu.obj
 0001:00004b10       _cpu_sample_on             10005b10 f   hprof_cpu.obj
 0001:00004c00       _cpu_sample_term           10005c00 f   hprof_cpu.obj
 0001:00004c90       ___local_stdio_printf_options 10005c90 f i hprof_error.obj
 0001:00004ca0       _debug_message             10005ca0 f   hprof_error.obj
 0001:00004cf0       _error_do_pause            10005cf0 f   hprof_error.obj
 0001:00004d40       _error_exit_process        10005d40 f   hprof_error.obj
 0001:00004d50       _error_handler             10005d50 f   hprof_error.obj
 0001:00004e30       _error_setup               10005e30 f   hprof_error.obj
 0001:00004eb0       _verbose_message           10005eb0 f   hprof_error.obj
 0001:00004f90       _event_call                10005f90 f   hprof_event.obj
 0001:00005060       _event_class_load          10006060 f   hprof_event.obj
 0001:00005200       _event_class_prepare       10006200 f   hprof_event.obj
 0001:00005260       _event_exception_catch     10006260 f   hprof_event.obj
 0001:000052c0       _event_newarray            100062c0 f   hprof_event.obj
 0001:00005320       _event_object_init         10006320 f   hprof_event.obj
 0001:00005380       _event_return              10006380 f   hprof_event.obj
 0001:00005460       _event_thread_end          10006460 f   hprof_event.obj
 0001:000054c0       _event_thread_start        100064c0 f   hprof_event.obj
 0001:00005610       _frame_cleanup             10006610 f   hprof_frame.obj
 0001:00005640       _frame_find_or_create      10006640 f   hprof_frame.obj
 0001:000056f0       _frame_get_location        100066f0 f   hprof_frame.obj
 0001:000057c0       _frame_get_status          100067c0 f   hprof_frame.obj
 0001:000057e0       _frame_init                100067e0 f   hprof_frame.obj
 0001:00005810       _frame_list                10006810 f   hprof_frame.obj
 0001:00005840       _frame_set_status          10006840 f   hprof_frame.obj
 0001:000058a0       _Agent_OnLoad@12           100068a0 f   hprof_init.obj
 0001:00005f50       _Agent_OnUnload@4          10006f50 f   hprof_init.obj
 0001:00007630       _fprintf                   10008630 f i hprof_init.obj
 0001:0000a1b0       _io_cleanup                1000b1b0 f   hprof_io.obj
 0001:0000a2c0       _io_flush                  1000b2c0 f   hprof_io.obj
 0001:0000a300       _io_heap_class_dump        1000b300 f   hprof_io.obj
 0001:0000a9b0       _io_heap_footer            1000b9b0 f   hprof_io.obj
 0001:0000aa00       _io_heap_header            1000ba00 f   hprof_io.obj
 0001:0000aa50       _io_heap_instance_dump     1000ba50 f   hprof_io.obj
 0001:0000ac60       _io_heap_object_array      1000bc60 f   hprof_io.obj
 0001:0000ad80       _io_heap_prim_array        1000bd80 f   hprof_io.obj
 0001:0000aeb0       _io_heap_root_java_frame   1000beb0 f   hprof_io.obj
 0001:0000af60       _io_heap_root_jni_global   1000bf60 f   hprof_io.obj
 0001:0000b000       _io_heap_root_jni_local    1000c000 f   hprof_io.obj
 0001:0000b0b0       _io_heap_root_monitor      1000c0b0 f   hprof_io.obj
 0001:0000b100       _io_heap_root_system_class 1000c100 f   hprof_io.obj
 0001:0000b160       _io_heap_root_thread       1000c160 f   hprof_io.obj
 0001:0000b1f0       _io_heap_root_thread_object 1000c1f0 f   hprof_io.obj
 0001:0000b2d0       _io_heap_root_unknown      1000c2d0 f   hprof_io.obj
 0001:0000b320       _io_setup                  1000c320 f   hprof_io.obj
 0001:0000b420       _io_write_class_load       1000c420 f   hprof_io.obj
 0001:0000b530       _io_write_class_unload     1000c530 f   hprof_io.obj
 0001:0000b5a0       _io_write_cpu_samples_elem 1000c5a0 f   hprof_io.obj
 0001:0000b690       _io_write_cpu_samples_footer 1000c690 f   hprof_io.obj
 0001:0000b6c0       _io_write_cpu_samples_header 1000c6c0 f   hprof_io.obj
 0001:0000b780       _io_write_file_header      1000c780 f   hprof_io.obj
 0001:0000ba10       _io_write_frame            1000ca10 f   hprof_io.obj
 0001:0000bb20       _io_write_heap_summary     1000cb20 f   hprof_io.obj
 0001:0000bc00       _io_write_monitor_dump_footer 1000cc00 f   hprof_io.obj
 0001:0000bc20       _io_write_monitor_dump_header 1000cc20 f   hprof_io.obj
 0001:0000bc40       _io_write_monitor_dump_state 1000cc40 f   hprof_io.obj
 0001:0000bda0       _io_write_monitor_dump_thread_state 1000cda0 f   hprof_io.obj
 0001:0000bfe0       _io_write_monitor_elem     1000cfe0 f   hprof_io.obj
 0001:0000c070       _io_write_monitor_footer   1000d070 f   hprof_io.obj
 0001:0000c090       _io_write_monitor_header   1000d090 f   hprof_io.obj
 0001:0000c100       _io_write_monitor_sleep    1000d100 f   hprof_io.obj
 0001:0000c170       _io_write_monitor_wait     1000d170 f   hprof_io.obj
 0001:0000c1e0       _io_write_monitor_waited   1000d1e0 f   hprof_io.obj
 0001:0000c250       _io_write_oldprof_elem     1000d250 f   hprof_io.obj
 0001:0000c310       _io_write_oldprof_header   1000d310 f   hprof_io.obj
 0001:0000c330       _io_write_sites_elem       1000d330 f   hprof_io.obj
 0001:0000c4e0       _io_write_sites_footer     1000d4e0 f   hprof_io.obj
 0001:0000c500       _io_write_sites_header     1000d500 f   hprof_io.obj
 0001:0000c670       _io_write_thread_end       1000d670 f   hprof_io.obj
 0001:0000c6f0       _io_write_thread_start     1000d6f0 f   hprof_io.obj
 0001:0000c870       _io_write_trace_elem       1000d870 f   hprof_io.obj
 0001:0000c980       _io_write_trace_header     1000d980 f   hprof_io.obj
 0001:0000d210       _ioname_cleanup            1000e210 f   hprof_ioname.obj
 0001:0000d240       _ioname_find_or_create     1000e240 f   hprof_ioname.obj
 0001:0000d280       _ioname_init               1000e280 f   hprof_ioname.obj
 0001:0000d2b0       _listener_init             1000e2b0 f   hprof_listener.obj
 0001:0000d740       _listener_term             1000e740 f   hprof_listener.obj
 0001:0000d950       _loader_cleanup            1000e950 f   hprof_loader.obj
 0001:0000d980       _loader_delete_global_references 1000e980 f   hprof_loader.obj
 0001:0000d9a0       _loader_find_or_create     1000e9a0 f   hprof_loader.obj
 0001:0000da70       _loader_init               1000ea70 f   hprof_loader.obj
 0001:0000daa0       _loader_list               1000eaa0 f   hprof_loader.obj
 0001:0000dad0       _loader_object_index       1000ead0 f   hprof_loader.obj
 0001:0000dc10       _DllMain@12                1000ec10 f   hprof_md.obj
 0001:0000dc80       __snprintf                 1000ec80 f i hprof_md.obj
 0001:0000dc80       _md_snprintf               1000ec80 f i hprof_md.obj
 0001:0000dcc0       _md_build_library_name     1000ecc0 f   hprof_md.obj
 0001:0000ddb0       _md_close                  1000edb0 f   hprof_md.obj
 0001:0000ddc0       _md_connect                1000edc0 f   hprof_md.obj
 0001:0000de70       _md_creat                  1000ee70 f   hprof_md.obj
 0001:0000de90       _md_creat_binary           1000ee90 f   hprof_md.obj
 0001:0000deb0       _md_find_library_entry     1000eeb0 f   hprof_md.obj
 0001:0000dec0       _md_get_microsecs          1000eec0 f   hprof_md.obj
 0001:0000ded0       _md_get_prelude_path       1000eed0 f   hprof_md.obj
 0001:0000df70       _md_get_thread_cpu_timemillis 1000ef70 f   hprof_md.obj
 0001:0000df70       _md_get_timemillis         1000ef70 f   hprof_md.obj
 0001:0000e020       _md_getpid                 1000f020 f   hprof_md.obj
 0001:0000e040       _md_htonl                  1000f040 f   hprof_md.obj
 0001:0000e050       _md_htons                  1000f050 f   hprof_md.obj
 0001:0000e060       _md_load_library           1000f060 f   hprof_md.obj
 0001:0000e150       _md_ntohl                  1000f150 f   hprof_md.obj
 0001:0000e160       _md_ntohs                  1000f160 f   hprof_md.obj
 0001:0000e170       _md_open                   1000f170 f   hprof_md.obj
 0001:0000e180       _md_open_binary            1000f180 f   hprof_md.obj
 0001:0000e1a0       _md_read                   1000f1a0 f   hprof_md.obj
 0001:0000e1b0       _md_recv                   1000f1b0 f   hprof_md.obj
 0001:0000e1d0       _md_seek                   1000f1d0 f   hprof_md.obj
 0001:0000e210       _md_send                   1000f210 f   hprof_md.obj
 0001:0000e230       _md_shutdown               1000f230 f   hprof_md.obj
 0001:0000e240       _md_sleep                  1000f240 f   hprof_md.obj
 0001:0000e250       _md_system_error           1000f250 f   hprof_md.obj
 0001:0000e2b0       _md_unload_library         1000f2b0 f   hprof_md.obj
 0001:0000e2c0       _md_vsnprintf              1000f2c0 f   hprof_md.obj
 0001:0000e300       _md_write                  1000f300 f   hprof_md.obj
 0001:0000e310       _sprintf                   1000f310 f i hprof_md.obj
 0001:0000e450       _monitor_cleanup           1000f450 f   hprof_monitor.obj
 0001:0000e480       _monitor_clear             1000f480 f   hprof_monitor.obj
 0001:0000e4a0       _monitor_contended_enter_event 1000f4a0 f   hprof_monitor.obj
 0001:0000e4f0       _monitor_contended_entered_event 1000f4f0 f   hprof_monitor.obj
 0001:0000e540       _monitor_init              1000f540 f   hprof_monitor.obj
 0001:0000e570       _monitor_list              1000f570 f   hprof_monitor.obj
 0001:0000e5a0       _monitor_wait_event        1000f5a0 f   hprof_monitor.obj
 0001:0000e650       _monitor_waited_event      1000f650 f   hprof_monitor.obj
 0001:0000e740       _monitor_write_contended_time 1000f740 f   hprof_monitor.obj
 0001:0000ea90       _object_cleanup            1000fa90 f   hprof_object.obj
 0001:0000eac0       _object_clear_references   1000fac0 f   hprof_object.obj
 0001:0000eae0       _object_free               1000fae0 f   hprof_object.obj
 0001:0000eb40       _object_get_kind           1000fb40 f   hprof_object.obj
 0001:0000eb70       _object_get_references     1000fb70 f   hprof_object.obj
 0001:0000eb90       _object_get_site           1000fb90 f   hprof_object.obj
 0001:0000ebc0       _object_get_size           1000fbc0 f   hprof_object.obj
 0001:0000ebf0       _object_get_thread_serial_number 1000fbf0 f   hprof_object.obj
 0001:0000ec10       _object_init               1000fc10 f   hprof_object.obj
 0001:0000ec50       _object_list               1000fc50 f   hprof_object.obj
 0001:0000ec80       _object_new                1000fc80 f   hprof_object.obj
 0001:0000ed60       _object_reference_dump     1000fd60 f   hprof_object.obj
 0001:0000eda0       _object_set_references     1000fda0 f   hprof_object.obj
 0001:0000edc0       _object_set_thread_serial_number 1000fdc0 f   hprof_object.obj
 0001:0000fa10       _reference_cleanup         10010a10 f   hprof_reference.obj
 0001:0000fa40       _reference_dump_class      10010a40 f   hprof_reference.obj
 0001:0000fa50       _reference_dump_instance   10010a50 f   hprof_reference.obj
 0001:0000fa60       _reference_init            10010a60 f   hprof_reference.obj
 0001:0000fa90       _reference_obj             10010a90 f   hprof_reference.obj
 0001:0000fb10       _reference_prim_array      10010b10 f   hprof_reference.obj
 0001:0000fba0       _reference_prim_field      10010ba0 f   hprof_reference.obj
 0001:000105b0       _site_cleanup              100115b0 f   hprof_site.obj
 0001:000105e0       _site_find_or_create       100115e0 f   hprof_site.obj
 0001:00010620       _site_get_class_index      10011620 f   hprof_site.obj
 0001:00010650       _site_get_trace_index      10011650 f   hprof_site.obj
 0001:00010680       _site_heapdump             10011680 f   hprof_site.obj
 0001:00010790       _site_init                 10011790 f   hprof_site.obj
 0001:000107c0       _site_list                 100117c0 f   hprof_site.obj
 0001:000107f0       _site_update_stats         100117f0 f   hprof_site.obj
 0001:00010890       _site_write                10011890 f   hprof_site.obj
 0001:00010b60       _stack_depth               10011b60 f   hprof_stack.obj
 0001:00010b70       _stack_element             10011b70 f   hprof_stack.obj
 0001:00010b80       _stack_init                10011b80 f   hprof_stack.obj
 0001:00010bd0       _stack_pop                 10011bd0 f   hprof_stack.obj
 0001:00010bf0       _stack_push                10011bf0 f   hprof_stack.obj
 0001:00010c90       _stack_term                10011c90 f   hprof_stack.obj
 0001:00010cb0       _stack_top                 10011cb0 f   hprof_stack.obj
 0001:00010cf0       _string_cleanup            10011cf0 f   hprof_string.obj
 0001:00010d20       _string_find_or_create     10011d20 f   hprof_string.obj
 0001:00010d60       _string_get                10011d60 f   hprof_string.obj
 0001:00010d90       _string_get_len            10011d90 f   hprof_string.obj
 0001:00010dc0       _string_init               10011dc0 f   hprof_string.obj
 0001:00010df0       _string_list               10011df0 f   hprof_string.obj
 0001:00011410       _table_cleanup             10012410 f   hprof_table.obj
 0001:00011560       _table_create_entry        10012560 f   hprof_table.obj
 0001:000115f0       _table_element_count       100125f0 f   hprof_table.obj
 0001:00011620       _table_find_entry          10012620 f   hprof_table.obj
 0001:00011690       _table_find_or_create_entry 10012690 f   hprof_table.obj
 0001:00011760       _table_free_entry          10012760 f   hprof_table.obj
 0001:00011890       _table_get_info            10012890 f   hprof_table.obj
 0001:00011920       _table_get_key             10012920 f   hprof_table.obj
 0001:000119c0       _table_initialize          100129c0 f   hprof_table.obj
 0001:00011af0       _table_lock_enter          10012af0 f   hprof_table.obj
 0001:00011b10       _table_lock_exit           10012b10 f   hprof_table.obj
 0001:00011b30       _table_walk_items          10012b30 f   hprof_table.obj
 0001:00011be0       _tag_class                 10012be0 f   hprof_tag.obj
 0001:00011ca0       _tag_create                10012ca0 f   hprof_tag.obj
 0001:00011cb0       _tag_extract               10012cb0 f   hprof_tag.obj
 0001:00011ce0       _tag_new_object            10012ce0 f   hprof_tag.obj
 0001:00012630       _tls_agent_thread          10013630 f   hprof_tls.obj
 0001:00012660       _tls_cleanup               10013660 f   hprof_tls.obj
 0001:00012690       _tls_clear_in_heap_dump    10013690 f   hprof_tls.obj
 0001:000126b0       _tls_delete_global_references 100136b0 f   hprof_tls.obj
 0001:000126d0       _tls_dump_monitor_state    100136d0 f   hprof_tls.obj
 0001:000128a0       _tls_dump_traces           100138a0 f   hprof_tls.obj
 0001:00012a00       _tls_find                  10013a00 f   hprof_tls.obj
 0001:00012a30       _tls_find_or_create        10013a30 f   hprof_tls.obj
 0001:00012b50       _tls_garbage_collect       10013b50 f   hprof_tls.obj
 0001:00012b90       _tls_get_in_heap_dump      10013b90 f   hprof_tls.obj
 0001:00012bb0       _tls_get_monitor           10013bb0 f   hprof_tls.obj
 0001:00012bd0       _tls_get_thread_serial_number 10013bd0 f   hprof_tls.obj
 0001:00012c10       _tls_get_trace             10013c10 f   hprof_tls.obj
 0001:00012d10       _tls_get_tracker_status    10013d10 f   hprof_tls.obj
 0001:00012df0       _tls_init                  10013df0 f   hprof_tls.obj
 0001:00012e20       _tls_list                  10013e20 f   hprof_tls.obj
 0001:00012e50       _tls_monitor_start_timer   10013e50 f   hprof_tls.obj
 0001:00012e80       _tls_monitor_stop_timer    10013e80 f   hprof_tls.obj
 0001:00012ec0       _tls_pop_exception_catch   10013ec0 f   hprof_tls.obj
 0001:00012fd0       _tls_pop_method            10013fd0 f   hprof_tls.obj
 0001:000130a0       _tls_push_method           100140a0 f   hprof_tls.obj
 0001:00013110       _tls_sample_all_threads    10014110 f   hprof_tls.obj
 0001:000131f0       _tls_set_in_heap_dump      100141f0 f   hprof_tls.obj
 0001:00013210       _tls_set_monitor           10014210 f   hprof_tls.obj
 0001:00013230       _tls_set_sample_status     10014230 f   hprof_tls.obj
 0001:00013260       _tls_set_thread_object_index 10014260 f   hprof_tls.obj
 0001:00013280       _tls_sum_sample_status     10014280 f   hprof_tls.obj
 0001:000132b0       _tls_thread_ended          100142b0 f   hprof_tls.obj
 0001:00013be0       _trace_cleanup             10014be0 f   hprof_trace.obj
 0001:00013c10       _trace_clear_cost          10014c10 f   hprof_trace.obj
 0001:00013c30       _trace_find_or_create      10014c30 f   hprof_trace.obj
 0001:00013c50       _trace_get_all_current     10014c50 f   hprof_trace.obj
 0001:00013d70       _trace_get_current         10014d70 f   hprof_trace.obj
 0001:00013e00       _trace_get_serial_number   10014e00 f   hprof_trace.obj
 0001:00013e20       _trace_increment_all_sample_costs 10014e20 f   hprof_trace.obj
 0001:00013fd0       _trace_increment_cost      10014fd0 f   hprof_trace.obj
 0001:00014030       _trace_init                10015030 f   hprof_trace.obj
 0001:00014060       _trace_list                10015060 f   hprof_trace.obj
 0001:00014090       _trace_output_cost         10015090 f   hprof_trace.obj
 0001:00014350       _trace_output_cost_in_prof_format 10015350 f   hprof_trace.obj
 0001:000145f0       _trace_output_unmarked     100155f0 f   hprof_trace.obj
 0001:00014a80       _tracker_disengage         10015a80 f   hprof_tracker.obj
 0001:00014a90       _tracker_engage            10015a90 f   hprof_tracker.obj
 0001:00014ab0       _tracker_method            10015ab0 f   hprof_tracker.obj
 0001:00014af0       _tracker_setup_class       10015af0 f   hprof_tracker.obj
 0001:00014b20       _tracker_setup_methods     10015b20 f   hprof_tracker.obj
 0001:00014ce0       _addCapabilities           10015ce0 f   hprof_util.obj
 0001:00015360       _createAgentThread         10016360 f   hprof_util.obj
 0001:00015650       _createRawMonitor          10016650 f   hprof_util.obj
 0001:000156a0       _deleteGlobalReference     100166a0 f   hprof_util.obj
 0001:000156c0       _deleteLocalReference      100166c0 f   hprof_util.obj
 0001:000156e0       _deleteWeakGlobalReference 100166e0 f   hprof_util.obj
 0001:00015700       _destroyRawMonitor         10016700 f   hprof_util.obj
 0001:00015740       _exceptionClear            10016740 f   hprof_util.obj
 0001:00015750       _exceptionDescribe         10016750 f   hprof_util.obj
 0001:00015760       _exceptionOccurred         10016760 f   hprof_util.obj
 0001:00015770       _findClass                 10016770 f   hprof_util.obj
 0001:000157f0       _followReferences          100167f0 f   hprof_util.obj
 0001:00015830       _getAllClassFieldInfo      10016830 f   hprof_util.obj
 0001:00015940       _getClassLoader            10016940 f   hprof_util.obj
 0001:00015990       _getClassSignature         10016990 f   hprof_util.obj
 0001:00015a20       _getClassStatus            10016a20 f   hprof_util.obj
 0001:00015a70       _getEnv                    10016a70 f   hprof_util.obj
 0001:00015b00       _getErrorName              10016b00 f   hprof_util.obj
 0001:00015b30       _getFrameCount             10016b30 f   hprof_util.obj
 0001:00015b60       _getJvmti                  10016b60 f   hprof_util.obj
 0001:00015d30       _getLineNumber             10016d30 f   hprof_util.obj
 0001:00015e80       _getLoadedClasses          10016e80 f   hprof_util.obj
 0001:00015ed0       _getMaxMemory              10016ed0 f   hprof_util.obj
 0001:000160c0       _getMethodClass            100170c0 f   hprof_util.obj
 0001:00016100       _getMethodID               10017100 f   hprof_util.obj
 0001:00016150       _getMethodName             10017150 f   hprof_util.obj
 0001:000161f0       _getObjectClass            100171f0 f   hprof_util.obj
 0001:00016210       _getObjectMonitorUsage     10017210 f   hprof_util.obj
 0001:00016250       _getObjectSize             10017250 f   hprof_util.obj
 0001:000162a0       _getOwnedMonitorInfo       100172a0 f   hprof_util.obj
 0001:00016300       _getPhase                  10017300 f   hprof_util.obj
 0001:00016330       _getPotentialCapabilities  10017330 f   hprof_util.obj
 0001:00016380       _getSourceFileName         10017380 f   hprof_util.obj
 0001:000163d0       _getStackTrace             100173d0 f   hprof_util.obj
 0001:00016410       _getStaticFieldID          10017410 f   hprof_util.obj
 0001:000164a0       _getStaticMethodID         100174a0 f   hprof_util.obj
 0001:00016530       _getSuperclass             10017530 f   hprof_util.obj
 0001:00016550       _getSystemProperty         10017550 f   hprof_util.obj
 0001:00016590       _getTag                    10017590 f   hprof_util.obj
 0001:000165e0       _getThreadGroupInfo        100175e0 f   hprof_util.obj
 0001:00016620       _getThreadInfo             10017620 f   hprof_util.obj
 0001:00016670       _getThreadListStackTraces  10017670 f   hprof_util.obj
 0001:000166c0       _getThreadLocalStorage     100176c0 f   hprof_util.obj
 0001:00016710       _getThreadState            10017710 f   hprof_util.obj
 0001:00016880       _hprof_free                10017880 f   hprof_util.obj
 0001:00016890       _hprof_malloc              10017890 f   hprof_util.obj
 0001:000168d0       _isMethodNative            100178d0 f   hprof_util.obj
 0001:00016910       _isSameObject              10017910 f   hprof_util.obj
 0001:00016940       _jvmtiAllocate             10017940 f   hprof_util.obj
 0001:000169a0       _jvmtiDeallocate           100179a0 f   hprof_util.obj
 0001:00016a80       _newGlobalReference        10017a80 f   hprof_util.obj
 0001:00016aa0       _newLocalReference         10017aa0 f   hprof_util.obj
 0001:00016ac0       _newWeakGlobalReference    10017ac0 f   hprof_util.obj
 0001:00016b40       _phaseString               10017b40 f   hprof_util.obj
 0001:00016ba0       _popLocalFrame             10017ba0 f   hprof_util.obj
 0001:00016be0       _primTypeToSigChar         10017be0 f   hprof_util.obj
 0001:00016c60       _pushLocalFrame            10017c60 f   hprof_util.obj
 0001:00016cf0       _rawMonitorEnter           10017cf0 f   hprof_util.obj
 0001:00016d30       _rawMonitorExit            10017d30 f   hprof_util.obj
 0001:00016d70       _rawMonitorNotifyAll       10017d70 f   hprof_util.obj
 0001:00016db0       _rawMonitorWait            10017db0 f   hprof_util.obj
 0001:00016df0       _registerNatives           10017df0 f   hprof_util.obj
 0001:00016e30       _runGC                     10017e30 f   hprof_util.obj
 0001:00016e70       _setEventCallbacks         10017e70 f   hprof_util.obj
 0001:00016eb0       _setEventNotificationMode  10017eb0 f   hprof_util.obj
 0001:00016ef0       _setStaticIntField         10017ef0 f   hprof_util.obj
 0001:00016f70       _setTag                    10017f70 f   hprof_util.obj
 0001:00016fb0       _setThreadLocalStorage     10017fb0 f   hprof_util.obj
 0001:00016ff0       _sigToPrimSize             10017ff0 f   hprof_util.obj
 0001:00017069       @__security_check_cookie@4 10018069 f   MSVCRT:secchk.obj
 0001:00017080       __alldiv                   10018080 f   MSVCRT:lldiv.obj
 0001:00017130       __allshr                   10018130 f   MSVCRT:llshr.obj
 0001:00017160       __ltod3                    10018160 f   MSVCRT:ftol3.obj
 0001:000174e1       __DllMainCRTStartup@12     100184e1 f   MSVCRT:dll_dllmain.obj
 0001:00017504       ___raise_securityfailure   10018504 f   MSVCRT:gs_report.obj
 0001:0001752c       ___report_gsfailure        1001852c f   MSVCRT:gs_report.obj
 0001:00017626       ___isa_available_init      10018626 f   MSVCRT:cpu_disp.obj
 0001:00017847       ___security_init_cookie    10018847 f   MSVCRT:gs_support.obj
 0001:00017892       ?__scrt_initialize_type_info@@YAXXZ 10018892 f   MSVCRT:tncleanup.obj
 0001:0001789e       ?__scrt_uninitialize_type_info@@YAXXZ 1001889e f   MSVCRT:tncleanup.obj
 0001:000178aa       ___local_stdio_scanf_options 100188aa f i MSVCRT:default_local_stdio_options.obj
 0001:000178b0       ___scrt_initialize_default_local_stdio_options 100188b0 f   MSVCRT:default_local_stdio_options.obj
 0001:00017911       ___scrt_acquire_startup_lock 10018911 f   MSVCRT:utility.obj
 0001:00017943       ___scrt_dllmain_after_initialize_c 10018943 f   MSVCRT:utility.obj
 0001:0001796e       ___scrt_dllmain_before_initialize_c 1001896e f   MSVCRT:utility.obj
 0001:0001797c       ___scrt_dllmain_crt_thread_attach 1001897c f   MSVCRT:utility.obj
 0001:0001799b       ___scrt_dllmain_crt_thread_detach 1001899b f   MSVCRT:utility.obj
 0001:000179a8       ___scrt_dllmain_exception_filter 100189a8 f   MSVCRT:utility.obj
 0001:000179dc       ___scrt_dllmain_uninitialize_c 100189dc f   MSVCRT:utility.obj
 0001:000179ff       ___scrt_dllmain_uninitialize_critical 100189ff f   MSVCRT:utility.obj
 0001:00017a0c       ___scrt_initialize_crt     10018a0c f   MSVCRT:utility.obj
 0001:00017a45       ___scrt_initialize_onexit_tables 10018a45 f   MSVCRT:utility.obj
 0001:00017acc       ___scrt_is_nonwritable_in_current_image 10018acc f   MSVCRT:utility.obj
 0001:00017b60       ___scrt_release_startup_lock 10018b60 f   MSVCRT:utility.obj
 0001:00017b7d       ___scrt_uninitialize_crt   10018b7d f   MSVCRT:utility.obj
 0001:00017ba5       ___scrt_get_dyn_tls_init_callback 10018ba5 f   MSVCRT:dyn_tls_init.obj
 0001:00017bab       ___scrt_fastfail           10018bab f   MSVCRT:utility_desktop.obj
 0001:00017cc6       __crt_debugger_hook        10018cc6 f   MSVCRT:utility_desktop.obj
 0001:00017cce       __RTC_Initialize           10018cce f   MSVCRT:initsect.obj
 0001:00017cfa       __RTC_Terminate            10018cfa f   MSVCRT:initsect.obj
 0001:00017d30       __SEH_prolog4              10018d30 f   MSVCRT:sehprolg4.obj
 0001:00017d75       __except_handler4          10018d75 f   MSVCRT:chandler4gs.obj
 0001:00017da4       __get_startup_argv_mode    10018da4 f   MSVCRT:argv_mode.obj
 0001:00017da8       ___scrt_is_ucrt_dll_in_use 10018da8 f   MSVCRT:ucrt_detection.obj
 0001:00017db4       _memcpy                    10018db4 f   vcruntime:VCRUNTIME140.dll
 0001:00017dba       _memset                    10018dba f   vcruntime:VCRUNTIME140.dll
 0001:00017dc0       _strrchr                   10018dc0 f   vcruntime:VCRUNTIME140.dll
 0001:00017dc6       _strchr                    10018dc6 f   vcruntime:VCRUNTIME140.dll
 0001:00017dcc       ___std_type_info_destroy_list 10018dcc f   vcruntime:VCRUNTIME140.dll
 0001:00017dd2       __except_handler4_common   10018dd2 f   vcruntime:VCRUNTIME140.dll
 0001:00017dd8       __initterm                 10018dd8 f   ucrt:api-ms-win-crt-runtime-l1-1-0.dll
 0001:00017dde       __initterm_e               10018dde f   ucrt:api-ms-win-crt-runtime-l1-1-0.dll
 0001:00017de4       __seh_filter_dll           10018de4 f   ucrt:api-ms-win-crt-runtime-l1-1-0.dll
 0001:00017dea       __configure_narrow_argv    10018dea f   ucrt:api-ms-win-crt-runtime-l1-1-0.dll
 0001:00017df0       __initialize_narrow_environment 10018df0 f   ucrt:api-ms-win-crt-runtime-l1-1-0.dll
 0001:00017df6       __initialize_onexit_table  10018df6 f   ucrt:api-ms-win-crt-runtime-l1-1-0.dll
 0001:00017dfc       __execute_onexit_table     10018dfc f   ucrt:api-ms-win-crt-runtime-l1-1-0.dll
 0001:00017e02       __cexit                    10018e02 f   ucrt:api-ms-win-crt-runtime-l1-1-0.dll
 0001:00017e08       ___acrt_initialize         10018e08 f   MSVCRT:ucrt_stubs.obj
 0001:00017e08       ___acrt_thread_attach      10018e08 f   MSVCRT:ucrt_stubs.obj
 0001:00017e08       ___acrt_thread_detach      10018e08 f   MSVCRT:ucrt_stubs.obj
 0001:00017e08       ___acrt_uninitialize       10018e08 f   MSVCRT:ucrt_stubs.obj
 0001:00017e08       ___acrt_uninitialize_critical 10018e08 f   MSVCRT:ucrt_stubs.obj
 0001:00017e08       ___scrt_stub_for_acrt_initialize 10018e08 f   MSVCRT:ucrt_stubs.obj
 0001:00017e08       ___scrt_stub_for_acrt_thread_attach 10018e08 f   MSVCRT:ucrt_stubs.obj
 0001:00017e08       ___scrt_stub_for_acrt_thread_detach 10018e08 f   MSVCRT:ucrt_stubs.obj
 0001:00017e08       ___scrt_stub_for_acrt_uninitialize 10018e08 f   MSVCRT:ucrt_stubs.obj
 0001:00017e08       ___scrt_stub_for_acrt_uninitialize_critical 10018e08 f   MSVCRT:ucrt_stubs.obj
 0001:00017e08       ___vcrt_initialize         10018e08 f   MSVCRT:ucrt_stubs.obj
 0001:00017e08       ___vcrt_thread_attach      10018e08 f   MSVCRT:ucrt_stubs.obj
 0001:00017e08       ___vcrt_thread_detach      10018e08 f   MSVCRT:ucrt_stubs.obj
 0001:00017e08       ___vcrt_uninitialize       10018e08 f   MSVCRT:ucrt_stubs.obj
 0001:00017e08       ___vcrt_uninitialize_critical 10018e08 f   MSVCRT:ucrt_stubs.obj
 0001:00017e0b       ___scrt_stub_for_is_c_termination_complete 10018e0b f   MSVCRT:ucrt_stubs.obj
 0001:00017e0b       __is_c_termination_complete 10018e0b f   MSVCRT:ucrt_stubs.obj
 0001:00017e0e       __filter_x86_sse2_floating_point_exception 10018e0e f   MSVCRT:x86_exception_filter.obj
 0001:00017e0e       __filter_x86_sse2_floating_point_exception_default 10018e0e f   MSVCRT:x86_exception_filter.obj
 0002:00000000       __imp__QueryPerformanceCounter@4 10019000     kernel32:KERNEL32.dll
 0002:00000004       __imp__IsDebuggerPresent@0 10019004     kernel32:KERNEL32.dll
 0002:00000008       __imp__InitializeSListHead@4 10019008     kernel32:KERNEL32.dll
 0002:0000000c       __imp__GetSystemTimeAsFileTime@4 1001900c     kernel32:KERNEL32.dll
 0002:00000010       __imp__GetCurrentThreadId@0 10019010     kernel32:KERNEL32.dll
 0002:00000014       __imp__GetCurrentProcessId@0 10019014     kernel32:KERNEL32.dll
 0002:00000018       __imp__IsProcessorFeaturePresent@4 10019018     kernel32:KERNEL32.dll
 0002:0000001c       __imp__TerminateProcess@8  1001901c     kernel32:KERNEL32.dll
 0002:00000020       __imp__GetCurrentProcess@0 10019020     kernel32:KERNEL32.dll
 0002:00000024       __imp__SetUnhandledExceptionFilter@4 10019024     kernel32:KERNEL32.dll
 0002:00000028       __imp__UnhandledExceptionFilter@4 10019028     kernel32:KERNEL32.dll
 0002:0000002c       __imp__SystemTimeToFileTime@8 1001902c     kernel32:KERNEL32.dll
 0002:00000030       __imp__FormatMessageA@28   10019030     kernel32:KERNEL32.dll
 0002:00000034       __imp__GetModuleFileNameA@12 10019034     kernel32:KERNEL32.dll
 0002:00000038       __imp__GetProcAddress@8    10019038     kernel32:KERNEL32.dll
 0002:0000003c       __imp__LoadLibraryA@4      1001903c     kernel32:KERNEL32.dll
 0002:00000040       __imp__GetLastError@0      10019040     kernel32:KERNEL32.dll
 0002:00000044       __imp__Sleep@4             10019044     kernel32:KERNEL32.dll
 0002:00000048       __imp__GetSystemTime@4     10019048     kernel32:KERNEL32.dll
 0002:0000004c       __imp__FreeLibrary@4       1001904c     kernel32:KERNEL32.dll
 0002:00000050       \177KERNEL32_NULL_THUNK_DATA 10019050     kernel32:KERNEL32.dll
 0002:00000054       __imp__memcpy              10019054     vcruntime:VCRUNTIME140.dll
 0002:00000058       __imp__memset              10019058     vcruntime:VCRUNTIME140.dll
 0002:0000005c       __imp____std_type_info_destroy_list 1001905c     vcruntime:VCRUNTIME140.dll
 0002:00000060       __imp__strchr              10019060     vcruntime:VCRUNTIME140.dll
 0002:00000064       __imp__strrchr             10019064     vcruntime:VCRUNTIME140.dll
 0002:00000068       __imp___except_handler4_common 10019068     vcruntime:VCRUNTIME140.dll
 0002:0000006c       \177VCRUNTIME140_NULL_THUNK_DATA 1001906c     vcruntime:VCRUNTIME140.dll
 0002:00000070       __imp__timeGetTime@0       10019070     winmm:WINMM.dll
 0002:00000074       \177WINMM_NULL_THUNK_DATA  10019074     winmm:WINMM.dll
 0002:00000078       __imp__ntohs@4             10019078     wsock32:WSOCK32.dll
 0002:0000007c       __imp__htons@4             1001907c     wsock32:WSOCK32.dll
 0002:00000080       __imp__htonl@4             10019080     wsock32:WSOCK32.dll
 0002:00000084       __imp__connect@12          10019084     wsock32:WSOCK32.dll
 0002:00000088       __imp__recv@16             10019088     wsock32:WSOCK32.dll
 0002:0000008c       __imp__send@16             1001908c     wsock32:WSOCK32.dll
 0002:00000090       __imp__closesocket@4       10019090     wsock32:WSOCK32.dll
 0002:00000094       __imp__shutdown@8          10019094     wsock32:WSOCK32.dll
 0002:00000098       __imp__socket@12           10019098     wsock32:WSOCK32.dll
 0002:0000009c       __imp__gethostbyname@4     1001909c     wsock32:WSOCK32.dll
 0002:000000a0       __imp__WSAStartup@8        100190a0     wsock32:WSOCK32.dll
 0002:000000a4       __imp__WSACleanup@0        100190a4     wsock32:WSOCK32.dll
 0002:000000a8       __imp__ntohl@4             100190a8     wsock32:WSOCK32.dll
 0002:000000ac       \177WSOCK32_NULL_THUNK_DATA 100190ac     wsock32:WSOCK32.dll
 0002:000000b0       __imp__strtod              100190b0     ucrt:api-ms-win-crt-convert-l1-1-0.dll
 0002:000000b4       __imp__strtol              100190b4     ucrt:api-ms-win-crt-convert-l1-1-0.dll
 0002:000000b8       \177api-ms-win-crt-convert-l1-1-0_NULL_THUNK_DATA 100190b8     ucrt:api-ms-win-crt-convert-l1-1-0.dll
 0002:000000bc       __imp__getenv              100190bc     ucrt:api-ms-win-crt-environment-l1-1-0.dll
 0002:000000c0       \177api-ms-win-crt-environment-l1-1-0_NULL_THUNK_DATA 100190c0     ucrt:api-ms-win-crt-environment-l1-1-0.dll
 0002:000000c4       __imp___access             100190c4     ucrt:api-ms-win-crt-filesystem-l1-1-0.dll
 0002:000000c8       __imp__remove              100190c8     ucrt:api-ms-win-crt-filesystem-l1-1-0.dll
 0002:000000cc       \177api-ms-win-crt-filesystem-l1-1-0_NULL_THUNK_DATA 100190cc     ucrt:api-ms-win-crt-filesystem-l1-1-0.dll
 0002:000000d0       __imp__free                100190d0     ucrt:api-ms-win-crt-heap-l1-1-0.dll
 0002:000000d4       __imp__malloc              100190d4     ucrt:api-ms-win-crt-heap-l1-1-0.dll
 0002:000000d8       \177api-ms-win-crt-heap-l1-1-0_NULL_THUNK_DATA 100190d8     ucrt:api-ms-win-crt-heap-l1-1-0.dll
 0002:000000dc       __imp___errno              100190dc     ucrt:api-ms-win-crt-runtime-l1-1-0.dll
 0002:000000e0       __imp___getpid             100190e0     ucrt:api-ms-win-crt-runtime-l1-1-0.dll
 0002:000000e0       __imp__getpid              100190e0     ucrt:api-ms-win-crt-runtime-l1-1-0.dll
 0002:000000e4       __imp__strerror            100190e4     ucrt:api-ms-win-crt-runtime-l1-1-0.dll
 0002:000000e8       __imp__signal              100190e8     ucrt:api-ms-win-crt-runtime-l1-1-0.dll
 0002:000000ec       __imp___cexit              100190ec     ucrt:api-ms-win-crt-runtime-l1-1-0.dll
 0002:000000f0       __imp___execute_onexit_table 100190f0     ucrt:api-ms-win-crt-runtime-l1-1-0.dll
 0002:000000f4       __imp__abort               100190f4     ucrt:api-ms-win-crt-runtime-l1-1-0.dll
 0002:000000f8       __imp__exit                100190f8     ucrt:api-ms-win-crt-runtime-l1-1-0.dll
 0002:000000fc       __imp___initterm           100190fc     ucrt:api-ms-win-crt-runtime-l1-1-0.dll
 0002:00000100       __imp___initterm_e         10019100     ucrt:api-ms-win-crt-runtime-l1-1-0.dll
 0002:00000104       __imp___seh_filter_dll     10019104     ucrt:api-ms-win-crt-runtime-l1-1-0.dll
 0002:00000108       __imp___configure_narrow_argv 10019108     ucrt:api-ms-win-crt-runtime-l1-1-0.dll
 0002:0000010c       __imp___initialize_narrow_environment 1001910c     ucrt:api-ms-win-crt-runtime-l1-1-0.dll
 0002:00000110       __imp___initialize_onexit_table 10019110     ucrt:api-ms-win-crt-runtime-l1-1-0.dll
 0002:00000114       \177api-ms-win-crt-runtime-l1-1-0_NULL_THUNK_DATA 10019114     ucrt:api-ms-win-crt-runtime-l1-1-0.dll
 0002:00000118       __imp____stdio_common_vsprintf 10019118     ucrt:api-ms-win-crt-stdio-l1-1-0.dll
 0002:0000011c       __imp___lseeki64           1001911c     ucrt:api-ms-win-crt-stdio-l1-1-0.dll
 0002:00000120       __imp____stdio_common_vfprintf 10019120     ucrt:api-ms-win-crt-stdio-l1-1-0.dll
 0002:00000124       __imp____acrt_iob_func     10019124     ucrt:api-ms-win-crt-stdio-l1-1-0.dll
 0002:00000128       __imp___write              10019128     ucrt:api-ms-win-crt-stdio-l1-1-0.dll
 0002:00000128       __imp__write               10019128     ucrt:api-ms-win-crt-stdio-l1-1-0.dll
 0002:0000012c       __imp___open               1001912c     ucrt:api-ms-win-crt-stdio-l1-1-0.dll
 0002:0000012c       __imp__open                1001912c     ucrt:api-ms-win-crt-stdio-l1-1-0.dll
 0002:00000130       __imp___read               10019130     ucrt:api-ms-win-crt-stdio-l1-1-0.dll
 0002:00000130       __imp__read                10019130     ucrt:api-ms-win-crt-stdio-l1-1-0.dll
 0002:00000134       \177api-ms-win-crt-stdio-l1-1-0_NULL_THUNK_DATA 10019134     ucrt:api-ms-win-crt-stdio-l1-1-0.dll
 0002:00000138       __imp__strtok_s            10019138     ucrt:api-ms-win-crt-string-l1-1-0.dll
 0002:0000013c       __imp__tolower             1001913c     ucrt:api-ms-win-crt-string-l1-1-0.dll
 0002:00000140       __imp__strncpy             10019140     ucrt:api-ms-win-crt-string-l1-1-0.dll
 0002:00000144       __imp___strdup             10019144     ucrt:api-ms-win-crt-string-l1-1-0.dll
 0002:00000144       __imp__strdup              10019144     ucrt:api-ms-win-crt-string-l1-1-0.dll
 0002:00000148       __imp__isprint             10019148     ucrt:api-ms-win-crt-string-l1-1-0.dll
 0002:0000014c       \177api-ms-win-crt-string-l1-1-0_NULL_THUNK_DATA 1001914c     ucrt:api-ms-win-crt-string-l1-1-0.dll
 0002:00000150       __imp___ctime64            10019150     ucrt:api-ms-win-crt-time-l1-1-0.dll
 0002:00000154       __imp___time64             10019154     ucrt:api-ms-win-crt-time-l1-1-0.dll
 0002:00000158       \177api-ms-win-crt-time-l1-1-0_NULL_THUNK_DATA 10019158     ucrt:api-ms-win-crt-time-l1-1-0.dll
 0002:0000015c       __imp__qsort               1001915c     ucrt:api-ms-win-crt-utility-l1-1-0.dll
 0002:00000160       \177api-ms-win-crt-utility-l1-1-0_NULL_THUNK_DATA 10019160     ucrt:api-ms-win-crt-utility-l1-1-0.dll
 0002:00000164       ___guard_check_icall_fptr  10019164     MSVCRT:guard_support.obj
 0002:00000168       ___castguard_check_failure_os_handled_fptr 10019168     MSVCRT:guard_support.obj
 0002:0000016c       ___xc_a                    1001916c     MSVCRT:initializers.obj
 0002:00000170       ___xc_z                    10019170     MSVCRT:initializers.obj
 0002:00000174       ___xi_a                    10019174     MSVCRT:initializers.obj
 0002:00000178       ___xi_z                    10019178     MSVCRT:initializers.obj
 0002:0000017c       ___xp_a                    1001917c     MSVCRT:initializers.obj
 0002:00000180       ___xp_z                    10019180     MSVCRT:initializers.obj
 0002:00000184       ___xt_a                    10019184     MSVCRT:initializers.obj
 0002:00000188       ___xt_z                    10019188     MSVCRT:initializers.obj
 0002:00000190       ??_C@_0BO@PPCEHAJA@Only?5part?5of?5buffer?5processed@ 10019190     hprof_check.obj
 0002:000001b0       ??_C@_0BP@KAJEFMEH@Unknown?5system?5error?5condition@ 100191b0     hprof_check.obj
 0002:000001d0       ??_C@_0BG@PMKOMKAJ@System?5?$CFs?5failed?3?5?$CFs?6@ 100191d0     hprof_check.obj
 0002:000001e8       ??_C@_0O@KBMJPJIE@hprof_check?4c@ 100191e8     hprof_check.obj
 0002:000001f8       ??_C@_05NGFEDHGN@write@    100191f8     hprof_check.obj
 0002:00000200       ??_C@_0BA@OIHJAJFL@bad?5type?5number@ 10019200     hprof_check.obj
 0002:00000210       ??_C@_06BJBFBFHM@0x?$CF08x@ 10019210     hprof_check.obj
 0002:00000218       ??_C@_06BEICJAKK@0x?$CF02x@ 10019218     hprof_check.obj
 0002:00000220       ??_C@_06BAAPOMBI@0x?$CF04x@ 10019220     hprof_check.obj
 0002:00000228       ??_C@_0L@MHPAILEE@0x?$CF04x?$CI?$CFc?$CJ@ 10019228     hprof_check.obj
 0002:00000234       ??_C@_06OAIHNJFH@?2u?$CF04x@ 10019234     hprof_check.obj
 0002:0000023c       ??_C@_02HAOIJKIC@?$CFc@    1001923c     hprof_check.obj
 0002:00000240       ??_C@_0L@GJLCDNL@0x?$CF08x?$CI?$CFf?$CJ@ 10019240     hprof_check.obj
 0002:0000024c       ??_C@_0P@KPOFLCNF@0x?$CF08x?$CF08x?$CI?$CFf?$CJ@ 1001924c     hprof_check.obj
 0002:0000025c       ??_C@_0L@FMEOCPGI@0x?$CF08x?$CF08x@ 1001925c     hprof_check.obj
 0002:00000268       ??_C@_06HPGEIPLA@?$DMnull?$DO@ 10019268     hprof_check.obj
 0002:00000270       ??_C@_01BJJEKLCA@?$CC@     10019270     hprof_check.obj
 0002:00000274       ??_C@_06FIJELGDL@?2x?$CF02x@ 10019274     hprof_check.obj
 0002:0000027c       ??_C@_06KEGKAONF@?$CFs0x?$CFx@ 1001927c     hprof_check.obj
 0002:00000284       ??_C@_08GKKHHGPJ@?$CFs0x?$CFx?9?$DO@ 10019284     hprof_check.obj
 0002:00000290       ??_C@_09HBBIIEJD@temp?5ctab@ 10019290     hprof_check.obj
 0002:0000029c       ??_C@_0BG@PHBGGCBG@HPROF_GC_ROOT_UNKNOWN@ 1001929c     hprof_check.obj
 0002:000002b4       ??_C@_0BJ@GDEKKILI@HPROF_GC_ROOT_JNI_GLOBAL@ 100192b4     hprof_check.obj
 0002:000002d0       ??_C@_0BI@ODPHJJBJ@HPROF_GC_ROOT_JNI_LOCAL@ 100192d0     hprof_check.obj
 0002:000002e8       ??_C@_0BJ@CPLOBCLD@HPROF_GC_ROOT_JAVA_FRAME@ 100192e8     hprof_check.obj
 0002:00000304       ??_C@_0BL@DJHFIEDF@HPROF_GC_ROOT_NATIVE_STACK@ 10019304     hprof_check.obj
 0002:00000320       ??_C@_0BL@JHEFKFML@HPROF_GC_ROOT_STICKY_CLASS@ 10019320     hprof_check.obj
 0002:0000033c       ??_C@_0BL@KEMDABPN@HPROF_GC_ROOT_THREAD_BLOCK@ 1001933c     hprof_check.obj
 0002:00000358       ??_C@_0BL@MMJBOEIG@HPROF_GC_ROOT_MONITOR_USED@ 10019358     hprof_check.obj
 0002:00000374       ??_C@_0BJ@BICPCHKK@HPROF_GC_ROOT_THREAD_OBJ@ 10019374     hprof_check.obj
 0002:00000390       ??_C@_0BE@GEIPHJMB@HPROF_GC_CLASS_DUMP@ 10019390     hprof_check.obj
 0002:000003a4       ??_C@_0BH@HIELBFJI@HPROF_GC_INSTANCE_DUMP@ 100193a4     hprof_check.obj
 0002:000003bc       ??_C@_0BI@NKGJEPHJ@HPROF_GC_OBJ_ARRAY_DUMP@ 100193bc     hprof_check.obj
 0002:000003d4       ??_C@_0BJ@CJBBPDCD@HPROF_GC_PRIM_ARRAY_DUMP@ 100193d4     hprof_check.obj
 0002:000003f0       ??_C@_07NFANNNEC@UNKNOWN@  100193f0     hprof_check.obj
 0002:000003f8       ??_C@_0BE@CBHNCPBK@H?$CD?$CFd?$EA?$CFd?5?$CFs?3?5ERROR?$CB?6@ 100193f8     hprof_check.obj
 0002:0000040c       ??_C@_0BJ@BOMKGAMF@unknown?5heap?5record?5type@ 1001940c     hprof_check.obj
 0002:00000428       ??_C@_0BB@PONDPCDE@p?$DN?$DNpstart?$CLnbytes@ 10019428     hprof_check.obj
 0002:0000043c       ??_C@_0BF@PECHNIEG@H?$CD?$CFd?$EA?$CFd?5?$CFs?3?5id?$DN0x?$CFx?6@ 1001943c     hprof_check.obj
 0002:00000454       ??_C@_0BP@PGHBFNMB@H?$CD?$CFd?$EA?$CFd?5?$CFs?3?5id?$DN0x?$CFx?0?5id2?$DN0x?$CFx?6@ 10019454     hprof_check.obj
 0002:00000474       ??_C@_0DE@GOLHEHCC@H?$CD?$CFd?$EA?$CFd?5?$CFs?3?5id?$DN0x?$CFx?0?5thread_ser@ 10019474     hprof_check.obj
 0002:000004a8       ??_C@_0CL@GNNONPMK@H?$CD?$CFd?$EA?$CFd?5?$CFs?3?5id?$DN0x?$CFx?0?5thread_ser@ 100194a8     hprof_check.obj
 0002:000004d8       ??_C@_0HC@LEKJFOKN@?$CItrace_serial_num?$CJ?5?$DO?$DN?5gdata?9?$DOtr@ 100194d8     hprof_check.obj
 0002:00000550       ??_C@_0EA@IHJEIELE@H?$CD?$CFd?$EA?$CFd?5?$CFs?3?5id?$DN0x?$CFx?0?5thread_ser@ 10019550     hprof_check.obj
 0002:00000590       ??_C@_0CK@CHDPPEIG@H?$CD?$CFd?$EA?$CFd?5?$CFs?3?5id?$DN0x?$CFx?0?5trace_seri@ 10019590     hprof_check.obj
 0002:000005bc       ??_C@_0DK@DLCBFCGK@?5?5su?$DN0x?$CFx?0?5ld?$DN0x?$CFx?0?5si?$DN0x?$CFx?0?5pr@ 100195bc     hprof_check.obj
 0002:000005f8       ??_C@_0BE@CFIFJJNL@?5?5instance_size?$DN?$CFd?6@ 100195f8     hprof_check.obj
 0002:0000060c       ??_C@_0CI@OPHKLNJG@?5?5constant_pool?5?$CFd?3?5cpi?$DN?$CFd?0?5ty?$DN@ 1001960c     hprof_check.obj
 0002:00000634       ??_C@_01EEMJAFIK@?6@       10019634     hprof_check.obj
 0002:00000638       ??_C@_0BJ@LJGJPBFI@?5?5static_field_count?$DN?$CFd?6@ 10019638     hprof_check.obj
 0002:00000654       ??_C@_0BE@BHOBLHPJ@?5?5static?5field?5?$CFd?3?5@ 10019654     hprof_check.obj
 0002:00000668       ??_C@_03LNKDLDCI@id?$DN@   10019668     hprof_check.obj
 0002:0000066c       ??_C@_0O@INODLMN@?0?5ty?$DN?$CFd?0?5val?$DN@ 1001966c     hprof_check.obj
 0002:0000067c       ??_C@_0BL@MLBLOLIO@?5?5instance_field_count?$DN?$CFd?6@ 1001967c     hprof_check.obj
 0002:00000698       ??_C@_0BG@LMBKGEEJ@?5?5instance_field?5?$CFd?3?5@ 10019698     hprof_check.obj
 0002:000006b0       ??_C@_08MLCDPIMM@?0?5ty?$DN?$CFd?6@ 100196b0     hprof_check.obj
 0002:000006bc       ??_C@_0DP@EAMBCAF@H?$CD?$CFd?$EA?$CFd?5?$CFs?3?5id?$DN0x?$CFx?0?5trace_seri@ 100196bc     hprof_check.obj
 0002:000006fc       ??_C@_0N@CGKPMCKK@?5?5field?5?$CFd?3?5@ 100196fc     hprof_check.obj
 0002:0000070c       ??_C@_0DP@KEJJKFNG@H?$CD?$CFd?$EA?$CFd?5?$CFs?3?5id?$DN0x?$CFx?0?5trace_seri@ 1001970c     hprof_check.obj
 0002:0000074c       ??_C@_0BB@GIMMJHDP@?5?5?$FL?$CFd?$FN?3?5id?$DN0x?$CFx?6@ 1001974c     hprof_check.obj
 0002:00000760       ??_C@_0DM@ELAFIGL@H?$CD?$CFd?$EA?$CFd?5?$CFs?3?5id?$DN0x?$CFx?0?5trace_seri@ 10019760     hprof_check.obj
 0002:0000079c       ??_C@_00CNPNBAHC@@         1001979c     hprof_check.obj
 0002:000007a0       ??_C@_08EKHGCGEE@?5?5val?$DN?$CFs@ 100197a0     hprof_check.obj
 0002:000007ac       ??_C@_04GCLKCGOG@?5?5?$CFs@ 100197ac     hprof_check.obj
 0002:000007b4       ??_C@_02MBJIFMOJ@?$CC?6@   100197b4     hprof_check.obj
 0002:000007b8       ??_C@_03OFAPEBGM@?$CFs?6@  100197b8     hprof_check.obj
 0002:000007bc       ??_C@_0BH@ODMGPLND@?6CHECK?5TAGS?3?5starting?6@ 100197bc     hprof_check.obj
 0002:000007d4       ??_C@_0O@DFBPNCDK@temp?5utf8?5map@ 100197d4     hprof_check.obj
 0002:000007e4       ??_C@_0L@OAOJOGOG@HPROF_UTF8@ 100197e4     hprof_check.obj
 0002:000007f0       ??_C@_0BL@PNFGFEBJ@size?$DO?$DN?$CIint?$CJsizeof?$CIHprofId?$CJ@ 100197f0     hprof_check.obj
 0002:0000080c       ??_C@_0CD@LIJOGBPJ@?$CD?$CFd?$EA?$CFd?3?5?$CFs?0?5sz?$DN?$CFd?0?5name_id?$DN0x?$CFx@ 1001980c     hprof_check.obj
 0002:00000830       ??_C@_0BB@ONOBIIEH@HPROF_LOAD_CLASS@ 10019830     hprof_check.obj
 0002:00000844       ??_C@_0CB@CAJECFPL@size?$DN?$DN2?$CK4?$CL2?$CK?$CIint?$CJsizeof?$CIHprofId@ 10019844     hprof_check.obj
 0002:00000868       ??_C@_0HC@MDOFHCCM@?$CIclass_serial_num?$CJ?5?$DO?$DN?5gdata?9?$DOcl@ 10019868     hprof_check.obj
 0002:000008e0       ??_C@_0FE@JEHKEEOG@?$CD?$CFd?$EA?$CFd?3?5?$CFs?0?5sz?$DN?$CFd?0?5class_serial@ 100198e0     hprof_check.obj
 0002:00000934       ??_C@_0BD@FFONNPAH@HPROF_UNLOAD_CLASS@ 10019934     hprof_check.obj
 0002:00000948       ??_C@_07MIJPMMAB@size?$DN?$DN4@ 10019948     hprof_check.obj
 0002:00000950       ??_C@_0CI@NCKLBDKC@?$CD?$CFd?$EA?$CFd?3?5?$CFs?0?5sz?$DN?$CFd?0?5class_serial@ 10019950     hprof_check.obj
 0002:00000978       ??_C@_0M@BGIACHM@HPROF_FRAME@ 10019978     hprof_check.obj
 0002:00000984       ??_C@_0CB@MNFOFHIB@size?$DN?$DN2?$CK4?$CL4?$CK?$CIint?$CJsizeof?$CIHprofId@ 10019984     hprof_check.obj
 0002:000009a8       ??_C@_0BE@HILIAEAK@?$CD?$CFd?$EA?$CFd?3?5?$CFs?0?5sz?$DN?$CFd?0?5@ 100199a8     hprof_check.obj
 0002:000009c0       ??_C@_0EM@NEDCOPAK@?5name_id?$DN0x?$CFx?0?5sig_id?$DN0x?$CFx?0?5sou@ 100199c0     hprof_check.obj
 0002:00000a0c       ??_C@_0M@EFOIIMOG@HPROF_TRACE@ 10019a0c     hprof_check.obj
 0002:00000a18       ??_C@_09BOHKANJD@size?$DO?$DN3?$CK4@ 10019a18     hprof_check.obj
 0002:00000a28       ??_C@_0EK@KCINGAKO@?$CD?$CFd?$EA?$CFd?3?5?$CFs?0?5sz?$DN?$CFd?0?5trace_serial@ 10019a28     hprof_check.obj
 0002:00000a74       ??_C@_05HHNKPPLF@0x?$CFx?0@ 10019a74     hprof_check.obj
 0002:00000a7c       ??_C@_02JODFHDIE@?$FN?6@   10019a7c     hprof_check.obj
 0002:00000a80       ??_C@_0BC@MFMDIHIE@HPROF_ALLOC_SITES@ 10019a80     hprof_check.obj
 0002:00000a94       ??_C@_0BA@LDLBGDDI@size?$DO?$DN2?$CL4?$CK4?$CL2?$CK8@ 10019a94     hprof_check.obj
 0002:00000aa8       ??_C@_0HB@HLMKAPIB@?$CD?$CFd?$EA?$CFd?3?5?$CFs?0?5sz?$DN?$CFd?0?5flags?$DN0x?$CFx?0?5@ 10019aa8     hprof_check.obj
 0002:00000b20       ??_C@_0GD@PEPAGFCM@?7?5?$CFd?3?5ty?$DN?$CFd?0?5class_serial_num?$DN?$CF@ 10019b20     hprof_check.obj
 0002:00000b84       ??_C@_0BD@IACOBOCN@HPROF_HEAP_SUMMARY@ 10019b84     hprof_check.obj
 0002:00000b98       ??_C@_0O@GBBJJLGJ@size?$DN?$DN2?$CK4?$CL2?$CK8@ 10019b98     hprof_check.obj
 0002:00000ba8       ??_C@_0EJ@MDCGLMNB@?$CD?$CFd?$EA?$CFd?3?5?$CFs?0?5sz?$DN?$CFd?0?5nblive?$DN?$CFd?0?5n@ 10019ba8     hprof_check.obj
 0002:00000bf4       ??_C@_0BD@OPDGIBFO@HPROF_START_THREAD@ 10019bf4     hprof_check.obj
 0002:00000c08       ??_C@_0HG@HCKHMBNJ@?$CIthread_serial_num?$CJ?5?$DO?$DN?5gdata?9?$DOt@ 10019c08     hprof_check.obj
 0002:00000c80       ??_C@_0EI@BIDIBGAO@?$CD?$CFd?$EA?$CFd?3?5?$CFs?0?5sz?$DN?$CFd?0?5thread_seria@ 10019c80     hprof_check.obj
 0002:00000cc8       ??_C@_03CPKFLABO@nm?$DN@   10019cc8     hprof_check.obj
 0002:00000ccc       ??_C@_0DB@GIJCGCMI@?5trace_serial_num?$DN?$CFu?0?5nm?$DN0x?$CFx?0?5@ 10019ccc     hprof_check.obj
 0002:00000d00       ??_C@_0BB@DAHLFMML@HPROF_END_THREAD@ 10019d00     hprof_check.obj
 0002:00000d14       ??_C@_0CJ@DGLABODG@?$CD?$CFd?$EA?$CFd?3?5?$CFs?0?5sz?$DN?$CFd?0?5thread_seria@ 10019d14     hprof_check.obj
 0002:00000d40       ??_C@_0BA@BJDLJLFF@HPROF_HEAP_DUMP@ 10019d40     hprof_check.obj
 0002:00000d50       ??_C@_0BK@ODPLGPKN@?$CD?$CFd?$EA?$CFd?3?5BEGIN?3?5?$CFs?0?5sz?$DN?$CFd?6@ 10019d50     hprof_check.obj
 0002:00000d6c       ??_C@_0CH@BHHAOIML@?$CD?$CFd?$EA?$CFd?3?5END?3?5?$CFs?0?5sz?$DN?$CFd?0?5nheap_r@ 10019d6c     hprof_check.obj
 0002:00000d94       ??_C@_0BI@CJBCMLBM@HPROF_HEAP_DUMP_SEGMENT@ 10019d94     hprof_check.obj
 0002:00000dac       ??_C@_0CC@ENEOELFC@?$CD?$CFd?$EA?$CFd?3?5BEGIN?5SEGMENT?3?5?$CFs?0?5sz?$DN?$CF@ 10019dac     hprof_check.obj
 0002:00000dd0       ??_C@_0CP@LFLJPIIL@?$CD?$CFd?$EA?$CFd?3?5END?5SEGMENT?3?5?$CFs?0?5sz?$DN?$CFd?0@ 10019dd0     hprof_check.obj
 0002:00000e00       ??_C@_0BE@KNNEDFKH@HPROF_HEAP_DUMP_END@ 10019e00     hprof_check.obj
 0002:00000e14       ??_C@_0CA@KNKMCKAJ@?$CD?$CFd?$EA?$CFd?3?5SEGMENT?5END?3?5?$CFs?0?5sz?$DN?$CFd?6@ 10019e14     hprof_check.obj
 0002:00000e34       ??_C@_0BC@HALEJIJE@HPROF_CPU_SAMPLES@ 10019e34     hprof_check.obj
 0002:00000e48       ??_C@_09KGMGGKPG@size?$DO?$DN2?$CK4@ 10019e48     hprof_check.obj
 0002:00000e54       ??_C@_0DF@MBJLKKLE@?$CD?$CFd?$EA?$CFd?3?5?$CFs?0?5sz?$DN?$CFd?0?5total_sample@ 10019e54     hprof_check.obj
 0002:00000e8c       ??_C@_0CH@MHBGMAD@?7?5?$CFd?3?5samples?$DN?$CFd?0?5trace_serial_@ 10019e8c     hprof_check.obj
 0002:00000eb4       ??_C@_0BH@ODPBMLKE@HPROF_CONTROL_SETTINGS@ 10019eb4     hprof_check.obj
 0002:00000ecc       ??_C@_09FCKBIKDF@size?$DN?$DN4?$CL2@ 10019ecc     hprof_check.obj
 0002:00000ed8       ??_C@_0CJ@BPPLJHCH@?$CD?$CFd?$EA?$CFd?3?5?$CFs?0?5sz?$DN?$CFd?0?5flags?$DN0x?$CFx?0?5@ 10019ed8     hprof_check.obj
 0002:00000f04       ??_C@_0BD@EHHNALKE@?$CD?$CFd?$EA?$CFd?3?5?$CFs?0?5sz?$DN?$CFd?6@ 10019f04     hprof_check.obj
 0002:00000f18       ??_C@_0BE@INEGKIJP@unknown?5record?5type@ 10019f18     hprof_check.obj
 0002:00000f2c       ??_C@_0BD@JKNLPFFK@p?$DM?$DN?$CIpstart?$CLnbytes?$CJ@ 10019f2c     hprof_check.obj
 0002:00000f40       ??_C@_0BD@HFIJEDLL@p?$DN?$DN?$CIpstart?$CLnbytes?$CJ@ 10019f40     hprof_check.obj
 0002:00000f54       ??_C@_05BPCDKMDE@fd?$DO?$DN0@ 10019f54     hprof_check.obj
 0002:00000f5c       ??_C@_0CA@MEEEFNIN@Cannot?5md_seek?$CI?$CJ?5to?5end?5of?5file@ 10019f5c     hprof_check.obj
 0002:00000f7c       ??_C@_0BD@JHIOCJLH@?$CI?$CIjint?$CJnbytes?$CJ?$DO512@ 10019f7c     hprof_check.obj
 0002:00000f90       ??_C@_0CC@MAKDCKBA@Cannot?5md_seek?$CI?$CJ?5to?5start?5of?5fi@ 10019f90     hprof_check.obj
 0002:00000fb4       ??_C@_0M@NLMPNCIE@image?$CB?$DNNULL@ 10019fb4     hprof_check.obj
 0002:00000fc0       ??_C@_0BE@IJINFLIE@System?5read?5failed?4@ 10019fc0     hprof_check.obj
 0002:00000fd4       ??_C@_0BG@NCGAHKKE@?$CI?$CIjint?$CJnbytes?$CJ?$DN?$DNnread@ 10019fd4     hprof_check.obj
 0002:00000fec       ??_C@_0BD@CIGAJKII@No?5file?5image?3?5?$CFs?6@ 10019fec     hprof_check.obj
 0002:00001000       ??_C@_0CD@CAODCGCP@strcmp?$CI?$CIchar?$CK?$CJp?0?5gdata?9?$DOheader?$CJ@ 1001a000     hprof_check.obj
 0002:00001024       ??_C@_0CF@GKEPBKCI@Filename?$DN?$CFs?0?5nbytes?$DN?$CFd?0?5header?$DN@ 1001a024     hprof_check.obj
 0002:0000104c       ??_C@_0BI@FKBBDLDN@idsize?$DN?$DNsizeof?$CIHprofId?$CJ@ 1001a04c     hprof_check.obj
 0002:00001064       ??_C@_0CF@FLGMMMCA@?$CD?$CFd?5total?5records?5found?5in?5?$CFd?5b@ 1001a064     hprof_check.obj
 0002:0000108c       ??_C@_0BD@HMGGFBMH@Ljava?1lang?1Object?$DL@ 1001a08c     hprof_class.obj
 0002:000010a0       ??_C@_0BH@PNGNOPN@Ljava?1io?1Serializable?$DL@ 1001a0a0     hprof_class.obj
 0002:000010b8       ??_C@_0BD@JFADHEFE@Ljava?1lang?1String?$DL@ 1001a0b8     hprof_class.obj
 0002:000010cc       ??_C@_0BC@JPHKFLAG@Ljava?1lang?1Class?$DL@ 1001a0cc     hprof_class.obj
 0002:000010e0       ??_C@_0BI@HIBJFPDC@Ljava?1lang?1ClassLoader?$DL@ 1001a0e0     hprof_class.obj
 0002:000010f8       ??_C@_0BD@HNGOJHNF@Ljava?1lang?1System?$DL@ 1001a0f8     hprof_class.obj
 0002:0000110c       ??_C@_0BD@KAGNMIPJ@Ljava?1lang?1Thread?$DL@ 1001a10c     hprof_class.obj
 0002:00001120       ??_C@_0BI@FKDHDBJA@Ljava?1lang?1ThreadGroup?$DL@ 1001a120     hprof_class.obj
 0002:00001138       ??_C@_0EB@DKDIJBO@0x?$CF08x?3?5Class?5?$CFs?0?5SN?$DN?$CFu?0?5status@ 1001a138     hprof_class.obj
 0002:0000117c       ??_C@_0CK@FBBIMDGA@?5?5?5?5Method?5?$CFd?3?5?$CC?$CFs?$CC?0?5sig?$DN?$CC?$CFs?$CC?0?5@ 1001a17c     hprof_class.obj
 0002:000011a8       ??_C@_05EKAMNAII@Class@    1001a1a8     hprof_class.obj
 0002:000011b0       ??_C@_0DM@BIDCIPNB@?9?9?9?9?9?9?9?9?9?9?9?9?9?9?9?9?9?9?9?9?9?5Class?5Tab@ 1001a1b0     hprof_class.obj
 0002:000011ec       ??_C@_0DM@LEMGKOFF@?9?9?9?9?9?9?9?9?9?9?9?9?9?9?9?9?9?9?9?9?9?9?9?9?9?9?9?9?9?9?9@ 1001a1ec     hprof_class.obj
 0002:00001228       ??_C@_0O@DLFKHHHD@hprof_class?4c@ 1001a228     hprof_class.obj
 0002:00001238       ??_C@_0CB@JLPJMIA@Cannot?5load?5class?5with?5findClas@ 1001a238     hprof_class.obj
 0002:0000125c       ??_C@_0CD@MOHADDFA@java?1lang?1IllegalArgumentExcept@ 1001a25c     hprof_class.obj
 0002:00001280       ??_C@_0DM@FGFCHEMJ@Could?5not?5find?5the?5java?1lang?1Il@ 1001a280     hprof_class.obj
 0002:000012bc       ??_C@_0N@NNAACLAO@Illegal?5mnum@ 1001a2bc     hprof_class.obj
 0002:000012cc       ??_C@_0P@BAGBBHBM@Name?5not?5found@ 1001a2cc     hprof_class.obj
 0002:000012dc       ??_C@_0CC@DOCAILJH@Missing?5jclass?5when?5fields?5need@ 1001a2dc     hprof_class.obj
 0002:00001300       ??_C@_0BE@NAHLKNGG@HPROF?5cpu?5loop?5lock@ 1001a300     hprof_cpu.obj
 0002:00001314       ??_C@_0BG@GHMBKHOC@HPROF?5cpu?5sample?5lock@ 1001a314     hprof_cpu.obj
 0002:0000132c       ??_C@_0BK@LKHEFACO@HPROF?5cpu?5sampling?5thread@ 1001a32c     hprof_cpu.obj
 0002:00001348       ??_C@_0BE@EFFKDDFJ@HPROF?5DUMPING?5CORE?6@ 1001a348     hprof_error.obj
 0002:0000135c       ??_C@_0CE@PHHBOMGP@HPROF?5SIGNAL?5?$CFd?5TERMINATED?5PROC@ 1001a35c     hprof_error.obj
 0002:00001380       ??_C@_0BK@LNMNOBI@HPROF?5TERMINATED?5PROCESS?6@ 1001a380     hprof_error.obj
 0002:0000139c       ??_C@_0BJ@ILCNEEPF@?6HPROF?5pause?5for?5PID?5?$CFd?6@ 1001a39c     hprof_error.obj
 0002:000013b8       ??_C@_0DB@GFACMNAF@?6?5HPROF?5pause?5got?5tired?5of?5wait@ 1001a3b8     hprof_error.obj
 0002:000013ec       ??_C@_0BC@HFMHFDPE@UnknownSourceFile@ 1001a3ec     hprof_error.obj
 0002:00001400       ??_C@_01OGPIMHDM@?$DP@     1001a400     hprof_error.obj
 0002:00001404       ??_C@_0CO@GDCCKAJE@HPROF?5ERROR?3?5?$CFs?5?$CIJVMTI?5Error?5?$CFs@ 1001a404     hprof_error.obj
 0002:00001434       ??_C@_0BJ@LNCNBLGB@HPROF?5ERROR?3?5?$CFs?5?$FL?$CFs?3?$CFd?$FN?6@ 1001a434     hprof_error.obj
 0002:00001450       ??_C@_0O@KAKNJEOI@hprof_event?4c@ 1001a450     hprof_event.obj
 0002:00001460       ??_C@_0O@NGGIEFHA@Illegal?5cnum?4@ 1001a460     hprof_event.obj
 0002:00001470       ??_C@_0EB@LGKGKPDH@Frame?50x?$CF08x?3?5method?$DN?$CFp?0?5locati@ 1001a470     hprof_frame.obj
 0002:000014b4       ??_C@_05MPDBFDHF@Frame@    1001a4b4     hprof_frame.obj
 0002:000014bc       ??_C@_0DM@HDIBGAFB@?9?9?9?9?9?9?9?9?9?9?9?9?9?9?9?9?9?9?9?9?9?5Frame?5Tab@ 1001a4bc     hprof_frame.obj
 0002:000014f8       ??_C@_0O@CMFFOGNE@java_crw_demo@ 1001a4f8     hprof_init.obj
 0002:00001508       ??_C@_0BC@GGCMOAGM@_java_crw_demo?$EA76@ 1001a508     hprof_init.obj
 0002:0000151c       ??_C@_0BI@NAKGBGBO@java_crw_demo_classname@ 1001a51c     hprof_init.obj
 0002:00001534       ??_C@_0BM@IDNEBGDK@_java_crw_demo_classname?$EA12@ 1001a534     hprof_init.obj
 0002:00001550       ??_C@_0L@NIPFOILE@?$CFs?5?$FL?$CFs?3?$CFd?$FN@ 1001a550     hprof_init.obj
 0002:0000155c       ??_C@_0N@IFEAIKFE@hprof_init?4c@ 1001a55c     hprof_init.obj
 0002:0000156c       ??_C@_0BE@FAJHFJE@invalid?5port?5number@ 1001a56c     hprof_init.obj
 0002:00001580       ??_C@_0BB@LCOFAJMA@hostname?5is?5NULL@ 1001a580     hprof_init.obj
 0002:00001594       ??_C@_04LCMACLFG@?4txt@    1001a594     hprof_init.obj
 0002:0000159c       ??_C@_07EMJMIMEK@?$CFs?4?$CFd?$CFs@ 1001a59c     hprof_init.obj
 0002:000015a4       ??_C@_01EANLCPLP@y@        1001a5a4     hprof_init.obj
 0002:000015a8       ??_C@_01EFFIKLCJ@n@        1001a5a8     hprof_init.obj
 0002:000015b0       ??_C@_0IDI@PKCEHLKG@?6?5?5?5?5?5HPROF?3?5Heap?5and?5CPU?5Profi@ 1001a5b0     hprof_init.obj
 0002:00001de8       ??_C@_05OCFCBLIP@hprof@    1001ade8     hprof_init.obj
 0002:00001df0       ??_C@_0BJ@NDAHLAI@?$CFs?5option?5error?3?5?$CFs?5?$CI?$CFs?$CJ@ 1001adf0     hprof_init.obj
 0002:00001e0c       ??_C@_04PCJFHION@help@     1001ae0c     hprof_init.obj
 0002:00001e14       ??_C@_0BE@GCMJIEKN@_JAVA_HPROF_OPTIONS@ 1001ae14     hprof_init.obj
 0002:00001e28       ??_C@_01IHBHIGKO@?0@       1001ae28     hprof_init.obj
 0002:00001e2c       ??_C@_0CF@KCMIGIIF@general?5syntax?5error?5parsing?5op@ 1001ae2c     hprof_init.obj
 0002:00001e54       ??_C@_04DAMGJPCA@file@     1001ae54     hprof_init.obj
 0002:00001e5c       ??_C@_0CM@FEEIPGCP@file?5or?5net?5options?5should?5only@ 1001ae5c     hprof_init.obj
 0002:00001e88       ??_C@_0CD@CGFHFHHF@syntax?5error?5parsing?5file?$DNfilen@ 1001ae88     hprof_init.obj
 0002:00001eac       ??_C@_03NBFOK@net@         1001aeac     hprof_init.obj
 0002:00001eb0       ??_C@_0BH@PJBFKPDJ@net?5option?5missing?5?8?3?8@ 1001aeb0     hprof_init.obj
 0002:00001ec8       ??_C@_0BI@IDICBEF@net?5option?5missing?5port@ 1001aec8     hprof_init.obj
 0002:00001ee0       ??_C@_06DLEPGFEF@format@   1001aee0     hprof_init.obj
 0002:00001ee8       ??_C@_0CA@EKAPMBCN@syntax?5error?5parsing?5format?$DNa?$HMb@ 1001aee8     hprof_init.obj
 0002:00001f08       ??_C@_01MCMALHOG@a@        1001af08     hprof_init.obj
 0002:00001f0c       ??_C@_01OJONOECF@b@        1001af0c     hprof_init.obj
 0002:00001f10       ??_C@_0CA@EMPDCICO@format?5option?5value?5must?5be?5a?$HMb@ 1001af10     hprof_init.obj
 0002:00001f30       ??_C@_05BJGJGKJC@depth@    1001af30     hprof_init.obj
 0002:00001f38       ??_C@_0CD@JBGECNOM@syntax?5error?5parsing?5depth?$DNDECI@ 1001af38     hprof_init.obj
 0002:00001f5c       ??_C@_0CM@CDCAOLHJ@depth?5option?5value?5must?5be?5deci@ 1001af5c     hprof_init.obj
 0002:00001f88       ??_C@_08CBFCMNKF@interval@ 1001af88     hprof_init.obj
 0002:00001f94       ??_C@_0CG@CJMKDEDE@syntax?5error?5parsing?5interval?$DND@ 1001af94     hprof_init.obj
 0002:00001fbc       ??_C@_0CO@DBLCEEJA@interval?5option?5value?5must?5be?5d@ 1001afbc     hprof_init.obj
 0002:00001fec       ??_C@_06JDMIDAGC@cutoff@   1001afec     hprof_init.obj
 0002:00001ff4       ??_C@_0CD@GGHCLFKF@syntax?5error?5parsing?5cutoff?$DNDOU@ 1001aff4     hprof_init.obj
 0002:00002018       ??_C@_0DE@MBFFIELL@cutoff?5option?5value?5must?5be?5flo@ 1001b018     hprof_init.obj
 0002:0000204c       ??_C@_03PBJBJNON@cpu@      1001b04c     hprof_init.obj
 0002:00002050       ??_C@_0CN@OJOLBMP@syntax?5error?5parsing?5cpu?$DNy?$HMsamp@ 1001b050     hprof_init.obj
 0002:00002080       ??_C@_07ODIFGGLK@samples@  1001b080     hprof_init.obj
 0002:00002088       ??_C@_05MJOOAIJH@times@    1001b088     hprof_init.obj
 0002:00002090       ??_C@_03PNKCFLFB@old@      1001b090     hprof_init.obj
 0002:00002094       ??_C@_0CN@KPFAPEKI@cpu?5option?5value?5must?5be?5y?$HMsamp@ 1001b094     hprof_init.obj
 0002:000020c4       ??_C@_04PKENOLLO@heap@     1001b0c4     hprof_init.obj
 0002:000020cc       ??_C@_0CJ@KEHGOHEP@syntax?5error?5parsing?5heap?$DNdump?$HM@ 1001b0cc     hprof_init.obj
 0002:000020f8       ??_C@_04GGLOKIEE@dump@     1001b0f8     hprof_init.obj
 0002:00002100       ??_C@_05PJPKCADK@sites@    1001b100     hprof_init.obj
 0002:00002108       ??_C@_03NFKEKGGK@all@      1001b108     hprof_init.obj
 0002:0000210c       ??_C@_0CJ@OPIHDONM@heap?5option?5value?5must?5be?5dump?$HM@ 1001b10c     hprof_init.obj
 0002:00002138       ??_C@_06ILKIAHNN@lineno@   1001b138     hprof_init.obj
 0002:00002140       ??_C@_0CA@LJGLHDND@lineno?5option?5value?5must?5be?5y?$HMn@ 1001b140     hprof_init.obj
 0002:00002160       ??_C@_06FJHNOCKE@thread@   1001b160     hprof_init.obj
 0002:00002168       ??_C@_0CA@IIGIIPGO@thread?5option?5value?5must?5be?5y?$HMn@ 1001b168     hprof_init.obj
 0002:00002188       ??_C@_03DBPOFDEI@doe@      1001b188     hprof_init.obj
 0002:0000218c       ??_C@_0BN@DCDFDPOH@doe?5option?5value?5must?5be?5y?$HMn@ 1001b18c     hprof_init.obj
 0002:000021ac       ??_C@_03DNKGIDNC@msa@      1001b1ac     hprof_init.obj
 0002:000021b0       ??_C@_0BN@IOIIIFGI@msa?5option?5value?5must?5be?5y?$HMn@ 1001b1b0     hprof_init.obj
 0002:000021d0       ??_C@_05BINPNAAL@force@    1001b1d0     hprof_init.obj
 0002:000021d8       ??_C@_0BP@BGDAHIEA@force?5option?5value?5must?5be?5y?$HMn@ 1001b1d8     hprof_init.obj
 0002:000021f8       ??_C@_07KBAMPNJK@verbose@  1001b1f8     hprof_init.obj
 0002:00002200       ??_C@_0CB@DLFJIIID@verbose?5option?5value?5must?5be?5y?$HM@ 1001b200     hprof_init.obj
 0002:00002224       ??_C@_0L@IPLLBFNC@primfields@ 1001b224     hprof_init.obj
 0002:00002230       ??_C@_0CE@NGFGIDIP@primfields?5option?5value?5must?5be@ 1001b230     hprof_init.obj
 0002:00002254       ??_C@_0L@BHFJHKGI@primarrays@ 1001b254     hprof_init.obj
 0002:00002260       ??_C@_0CE@KKEDLIMN@primarrays?5option?5value?5must?5be@ 1001b260     hprof_init.obj
 0002:00002284       ??_C@_07LAMOHCEE@monitor@  1001b284     hprof_init.obj
 0002:0000228c       ??_C@_0CB@MBCCNCCN@monitor?5option?5value?5must?5be?5y?$HM@ 1001b28c     hprof_init.obj
 0002:000022b0       ??_C@_07EHNIJGFI@gc_okay@  1001b2b0     hprof_init.obj
 0002:000022b8       ??_C@_0CB@JPJMDDAJ@gc_okay?5option?5value?5must?5be?5y?$HM@ 1001b2b8     hprof_init.obj
 0002:000022dc       ??_C@_08KMAEEIGA@logflags@ 1001b2dc     hprof_init.obj
 0002:000022e8       ??_C@_0CG@DPIOJAEB@logflags?5option?5value?5must?5be?5n@ 1001b2e8     hprof_init.obj
 0002:00002310       ??_C@_0L@NDPADBNN@debugflags@ 1001b310     hprof_init.obj
 0002:0000231c       ??_C@_0CI@IHAKJFIH@debugflags?5option?5value?5must?5be@ 1001b31c     hprof_init.obj
 0002:00002344       ??_C@_08JHOBLGK@coredump@  1001b344     hprof_init.obj
 0002:00002350       ??_C@_0CC@HFBDFNIP@coredump?5option?5value?5must?5be?5y@ 1001b350     hprof_init.obj
 0002:00002374       ??_C@_09KOPDMKB@exitpause@ 1001b374     hprof_init.obj
 0002:00002380       ??_C@_0DM@FNMJKPHI@The?5exitpause?5option?5was?5remove@ 1001b380     hprof_init.obj
 0002:000023bc       ??_C@_09NDIDIJNG@errorexit@ 1001b3bc     hprof_init.obj
 0002:000023c8       ??_C@_0CD@CBEHPELG@errorexit?5option?5value?5must?5be?5@ 1001b3c8     hprof_init.obj
 0002:000023ec       ??_C@_05PDJBBECF@pause@    1001b3ec     hprof_init.obj
 0002:000023f4       ??_C@_0BP@IGBDALOK@pause?5option?5value?5must?5be?5y?$HMn@ 1001b3f4     hprof_init.obj
 0002:00002414       ??_C@_05GFCDIDHO@debug@    1001b414     hprof_init.obj
 0002:0000241c       ??_C@_0BP@OHLBFOK@debug?5option?5value?5must?5be?5y?$HMn@ 1001b41c     hprof_init.obj
 0002:0000243c       ??_C@_08KLNFLELA@precrash@ 1001b43c     hprof_init.obj
 0002:00002448       ??_C@_0ED@JHBHPMON@The?5precrash?5option?5was?5removed@ 1001b448     hprof_init.obj
 0002:0000248c       ??_C@_01MMEEDKFM@X@        1001b48c     hprof_init.obj
 0002:00002490       ??_C@_0BP@DMEMBFPB@X?5option?5value?5must?5be?5numeric@ 1001b490     hprof_init.obj
 0002:000024b0       ??_C@_0BB@BKPNNECG@Unknown?5option?3?5@ 1001b4b0     hprof_init.obj
 0002:000024c4       ??_C@_0CN@DNEGEHLK@cpu?$DNtimes?$HMold?5is?5not?5supported?5@ 1001b4c4     hprof_init.obj
 0002:000024f4       ??_C@_0CJ@GDLIPKLO@monitor?$DNy?5is?5not?5supported?5with@ 1001b4f4     hprof_init.obj
 0002:00002520       ??_C@_0L@LEDDPCIJ@java?4hprof@ 1001b520     hprof_init.obj
 0002:0000252c       ??_C@_0P@JFGLGPBO@java?4hprof?4txt@ 1001b52c     hprof_init.obj
 0002:0000253c       ??_C@_04MBLKECLF@?4TMP@    1001b53c     hprof_init.obj
 0002:00002544       ??_C@_0L@FGICFCIH@?4check?4txt@ 1001b544     hprof_init.obj
 0002:00002550       ??_C@_0CA@OKBAMGHH@can?8t?5create?5temp?5heap?5file?3?5?$CFs@ 1001b550     hprof_init.obj
 0002:00002570       ??_C@_0BH@GNMJDGKG@can?8t?5connect?5to?5?$CFs?3?$CFu@ 1001b570     hprof_init.obj
 0002:00002588       ??_C@_0BO@MBPIAAPH@can?8t?5create?5profile?5file?3?5?$CFs@ 1001b588     hprof_init.obj
 0002:000025a8       ??_C@_07OKDJEMIF@Dumping@  1001b5a8     hprof_init.obj
 0002:000025b0       ??_C@_0BN@OCIBMNDP@?5contended?5monitor?5usage?5?4?4?4@ 1001b5b0     hprof_init.obj
 0002:000025d0       ??_C@_0P@BENJNADH@?5Java?5heap?5?4?4?4@ 1001b5d0     hprof_init.obj
 0002:000025e0       ??_C@_0BG@BLJMODIC@?5allocation?5sites?5?4?4?4@ 1001b5e0     hprof_init.obj
 0002:000025f8       ??_C@_0CL@JCIEPIKM@?5CPU?5usage?5by?5sampling?5running?5@ 1001b5f8     hprof_init.obj
 0002:00002624       ??_C@_0CB@PKCDBGOG@?5CPU?5usage?5by?5timing?5methods?5?4?4@ 1001b624     hprof_init.obj
 0002:00002648       ??_C@_0CC@LHKHFDOC@?5CPU?5usage?5in?5old?5prof?5format?5?4@ 1001b648     hprof_init.obj
 0002:0000266c       ??_C@_07HDGNKME@?5done?4?6@ 1001b66c     hprof_init.obj
 0002:00002674       ??_C@_0BD@NGKJFPEL@JAVA?5PROFILE?51?40?41@ 1001b674     hprof_init.obj
 0002:00002688       ??_C@_0BD@PNIEAMII@JAVA?5PROFILE?51?40?42@ 1001b688     hprof_init.obj
 0002:0000269c       ??_C@_0BI@OCGOOHFN@HPROF?5gc_finish?5watcher@ 1001b69c     hprof_init.obj
 0002:000026b4       ??_C@_0BI@PEEGGNOL@VM?5Death?5during?5VM?5Init@ 1001b6b4     hprof_init.obj
 0002:000026cc       ??_C@_0BI@ILJEGKOI@VM?5Death?5before?5VM?5Init@ 1001b6cc     hprof_init.obj
 0002:000026e4       ??_C@_0BJ@PGHAIEAL@VM?5Death?5more?5than?5once?$DP@ 1001b6e4     hprof_init.obj
 0002:00002700       ??_C@_0BK@PFEIMFJI@No?5classname?5in?5classfile@ 1001b700     hprof_init.obj
 0002:0000271c       ??_C@_0BK@CJJFDDOP@Ran?5out?5of?5malloc?$CI?$CJ?5space@ 1001b71c     hprof_init.obj
 0002:00002738       ??_C@_0CB@MLGJILKK@com?1sun?1demo?1jvmti?1hprof?1Tracke@ 1001b738     hprof_init.obj
 0002:0000275c       ??_C@_0BG@JLFLBLJI@?$CILjava?1lang?1Object?$DL?$CJV@ 1001b75c     hprof_init.obj
 0002:00002774       ??_C@_08IPKKBCGH@NewArray@ 1001b774     hprof_init.obj
 0002:00002780       ??_C@_0L@PNDODNGI@ObjectInit@ 1001b780     hprof_init.obj
 0002:0000278c       ??_C@_05MNEAHDDF@?$CIII?$CJV@ 1001b78c     hprof_init.obj
 0002:00002794       ??_C@_0L@PBHNBFDL@ReturnSite@ 1001b794     hprof_init.obj
 0002:000027a0       ??_C@_08KDGHMPPK@CallSite@ 1001b7a0     hprof_init.obj
 0002:000027ac       ??_C@_0CD@OELEBCJC@Lcom?1sun?1demo?1jvmti?1hprof?1Track@ 1001b7ac     hprof_init.obj
 0002:000027d0       ??_C@_0BG@HAHGGNHO@sun?4boot?4library?4path@ 1001b7d0     hprof_init.obj
 0002:000027e8       ??_C@_0BH@BEIPEIGO@Could?5not?5find?5library@ 1001b7e8     hprof_init.obj
 0002:00002800       ??_C@_0CA@IAAIIKKH@Cannot?5find?5library?5symbol?5?8?$CFs?8@ 1001b800     hprof_init.obj
 0002:00002820       ??_C@_0FP@EEPNNOPI@Cannot?5load?5this?5JVM?5TI?5agent?5t@ 1001b820     hprof_init.obj
 0002:00002880       ??_C@_03BKOAHEHB@npt@      1001b880     hprof_init.obj
 0002:00002884       ??_C@_0BL@HCOIICMK@Could?5not?5find?5npt?5library@ 1001b884     hprof_init.obj
 0002:000028a0       ??_C@_0BA@GOCLFPKI@NptEnv?$CK?5is?5NULL@ 1001b8a0     hprof_init.obj
 0002:000028b0       ??_C@_0P@KEJEBKCF@NPT?5ERROR?3?5?$CFs?6@ 1001b8b0     hprof_init.obj
 0002:000028c0       ??_C@_0BE@PIBOIGHP@Cannot?5open?5library@ 1001b8c0     hprof_init.obj
 0002:000028d4       ??_C@_0O@MIMNKEMK@nptInitialize@ 1001b8d4     hprof_init.obj
 0002:000028e4       ??_C@_0BK@HOJGHELP@Cannot?5find?5nptInitialize@ 1001b8e4     hprof_init.obj
 0002:00002900       ??_C@_05CJAIGNCM@0?40?40@  1001b900     hprof_init.obj
 0002:00002908       ??_C@_0BJ@BCAAKKFG@Cannot?5initialize?5NptEnv@ 1001b908     hprof_init.obj
 0002:00002924       ??_C@_0BI@KDIGKBKK@Cannot?5load?5npt?5library@ 1001b924     hprof_init.obj
 0002:0000293c       ??_C@_0CE@MEIGLHJ@Cannot?5initialize?5npt?5utf?5funct@ 1001b93c     hprof_init.obj
 0002:00002960       ??_C@_0BA@PEOHBHKP@HPROF?5dump?5lock@ 1001b960     hprof_init.obj
 0002:00002970       ??_C@_0BH@JAOAIHPM@HPROF?5data?5access?5lock@ 1001b970     hprof_init.obj
 0002:00002988       ??_C@_0BE@BAHELICG@HPROF?5callback?5lock@ 1001b988     hprof_init.obj
 0002:0000299c       ??_C@_0BF@GNHLLGIJ@HPROF?5callback?5block@ 1001b99c     hprof_init.obj
 0002:000029b4       ??_C@_0BH@PHBLECPG@HPROF?5object?5free?5lock@ 1001b9b4     hprof_init.obj
 0002:000029cc       ??_C@_0BF@ILMDJCHH@HPROF?5gc_finish?5lock@ 1001b9cc     hprof_init.obj
 0002:000029e8       __real@3f1a36e2eb1c432d    1001b9e8     hprof_init.obj
 0002:000029f0       ??_C@_0O@IFNENBMK@Unknown_class@ 1001b9f0     hprof_io.obj
 0002:00002a00       ??_C@_0P@DHLBOJDB@Unknown_method@ 1001ba00     hprof_io.obj
 0002:00002a10       ??_C@_02HCKGKOFO@?$CI?$CJ@ 1001ba10     hprof_io.obj
 0002:00002a14       ??_C@_04IHGKJMLH@byte@     1001ba14     hprof_io.obj
 0002:00002a1c       ??_C@_04ENMBGAPA@char@     1001ba1c     hprof_io.obj
 0002:00002a24       ??_C@_04DBJPMPLO@enum@     1001ba24     hprof_io.obj
 0002:00002a2c       ??_C@_05KNFBNCOH@float@    1001ba2c     hprof_io.obj
 0002:00002a34       ??_C@_06BNJCAIGJ@double@   1001ba34     hprof_io.obj
 0002:00002a3c       ??_C@_03JBIPMCLC@int@      1001ba3c     hprof_io.obj
 0002:00002a40       ??_C@_04GOKPGOLB@long@     1001ba40     hprof_io.obj
 0002:00002a48       ??_C@_05BFKKPKCG@short@    1001ba48     hprof_io.obj
 0002:00002a50       ??_C@_04GKJNKENE@void@     1001ba50     hprof_io.obj
 0002:00002a58       ??_C@_07GOBOHMJA@boolean@  1001ba58     hprof_io.obj
 0002:00002a60       ??_C@_0L@MBGCIHKI@hprof_io?4c@ 1001ba60     hprof_io.obj
 0002:00002a6c       ??_C@_04MIIPNNEF@send@     1001ba6c     hprof_io.obj
 0002:00002a74       ??_C@_0M@MIOILAFG@?5thread?5?$CFd?0@ 1001ba74     hprof_io.obj
 0002:00002a80       ??_C@_0L@NDJLKNB@?5thread?5?$CFd@ 1001ba80     hprof_io.obj
 0002:00002a8c       ??_C@_0BD@IAMJIPJO@?5?$DMunknown?5thread?$DO?0@ 1001ba8c     hprof_io.obj
 0002:00002aa0       ??_C@_0BC@JODADJHG@?5?$DMunknown?5thread?$DO@ 1001baa0     hprof_io.obj
 0002:00002ab4       ??_C@_0O@PMAAFLKH@jvm?4hprof?4txt@ 1001bab4     hprof_io.obj
 0002:00002ac4       ??_C@_0O@NCFAOBDD@Can?8t?5open?5?$CFs@ 1001bac4     hprof_io.obj
 0002:00002ad4       ??_C@_0BA@CADMPAOC@?$CFs?0?5created?5?$CFs?6@ 1001bad4     hprof_io.obj
 0002:00002ae4       ??_C@_04POLDLDMI@read@     1001bae4     hprof_io.obj
 0002:00002aec       ??_C@_0M@BFCDGIM@?6?9?9?9?9?9?9?9?9?6?6@ 1001baec     hprof_io.obj
 0002:00002af8       ??_C@_0BP@CLCGNIMI@SITES?5BEGIN?5?$CIordered?5by?5?$CFs?$CJ?5?$CFs@ 1001baf8     hprof_io.obj
 0002:00002b18       ??_C@_0EA@CFBHFKDL@?5?5?5?5?5?5?5?5?5?5percent?5?5?5?5?5?5?5?5?5?5live@ 1001bb18     hprof_io.obj
 0002:00002b58       ??_C@_0DP@EOEKDJEO@?5rank?5?5?5self?5?5accum?5?5?5?5?5bytes?5o@ 1001bb58     hprof_io.obj
 0002:00002b98       ??_C@_0CM@CBLHKJFI@?$CF5u?5?$CF5?42f?$CF?$CF?5?$CF5?42f?$CF?$CF?5?$CF9u?5?$CF4u?5?$CF9u@ 1001bb98     hprof_io.obj
 0002:00002bc4       ??_C@_0L@CKHNMGBC@SITES?5END?6@ 1001bbc4     hprof_io.obj
 0002:00002bd0       ??_C@_0DH@NGILCPCO@THREAD?5START?5?$CIobj?$DN?$CFx?0?5id?5?$DN?5?$CFd?0?5@ 1001bbd0     hprof_io.obj
 0002:00002c08       ??_C@_0BG@PIAADDAB@THREAD?5END?5?$CIid?5?$DN?5?$CFd?$CJ?6@ 1001bc08     hprof_io.obj
 0002:00002c20       ??_C@_09BONBOKMJ@TRACE?5?$CFu?3@ 1001bc20     hprof_io.obj
 0002:00002c2c       ??_C@_0N@OMDMKKMG@?5?$CIthread?$DN?$CFd?$CJ@ 1001bc2c     hprof_io.obj
 0002:00002c3c       ??_C@_0BI@FDDGHNEP@?5?$CIfrom?5?$CFs?5phase?5of?5JVM?$CJ@ 1001bc3c     hprof_io.obj
 0002:00002c54       ??_C@_09JPFCIILH@?7?$DMempty?$DO?6@ 1001bc54     hprof_io.obj
 0002:00002c60       ??_C@_0BA@KBBHNEBH@Compiled?5method@ 1001bc60     hprof_io.obj
 0002:00002c70       ??_C@_0O@GNIBGOFH@Native?5method@ 1001bc70     hprof_io.obj
 0002:00002c80       ??_C@_0N@CANDBIMJ@Unknown?5line@ 1001bc80     hprof_io.obj
 0002:00002c90       ??_C@_02DPKJAMEF@?$CFd@    1001bc90     hprof_io.obj
 0002:00002c94       ??_C@_0BB@EPPOLNMC@?$DMUnknown?5Method?$DO@ 1001bc94     hprof_io.obj
 0002:00002ca8       ??_C@_0BB@CIKHEIJM@?$DMUnknown?5Source?$DO@ 1001bca8     hprof_io.obj
 0002:00002cbc       ??_C@_0P@EGBEGAHH@?7?$CFs?4?$CFs?$CI?$CFs?3?$CFs?$CJ?6@ 1001bcbc     hprof_io.obj
 0002:00002ccc       ??_C@_0M@OCKALELD@CPU?5SAMPLES@ 1001bccc     hprof_io.obj
 0002:00002cd8       ??_C@_0O@HDJHNIOL@CPU?5TIME?5?$CIms?$CJ@ 1001bcd8     hprof_io.obj
 0002:00002ce8       ??_C@_0BJ@MCGJLPEC@?$CFs?5BEGIN?5?$CItotal?5?$DN?5?$CFd?$CJ?5?$CFs@ 1001bce8     hprof_io.obj
 0002:00002d04       ??_C@_0CJ@FEPGPPDL@rank?5?5?5self?5?5accum?5?5?5count?5trac@ 1001bd04     hprof_io.obj
 0002:00002d30       ??_C@_0BM@MJAPPKNB@?$CF4u?5?$CF5?42f?$CF?$CF?5?$CF5?42f?$CF?$CF?5?$CF7u?5?$CF5u@ 1001bd30     hprof_io.obj
 0002:00002d4c       ??_C@_07DGNNNLHO@?5?$CFs?4?$CFs?6@ 1001bd4c     hprof_io.obj
 0002:00002d54       ??_C@_0BA@LIKBLINJ@?5?$DMempty?5trace?$DO?6@ 1001bd54     hprof_io.obj
 0002:00002d64       ??_C@_07JHMDLGIF@?$CFs?5END?6@ 1001bd64     hprof_io.obj
 0002:00002d6c       ??_C@_0BK@IEECFLPB@count?5callee?5caller?5time?6@ 1001bd6c     hprof_io.obj
 0002:00002d88       ??_C@_03JDANDILB@?$CFd?5@  1001bd88     hprof_io.obj
 0002:00002d8c       ??_C@_08NBABFLDC@?$CFs?4?$CFs?$CFs?5@ 1001bd8c     hprof_io.obj
 0002:00002d98       ??_C@_0BB@DEAIDOKN@?$DMunknown?5callee?$DO@ 1001bd98     hprof_io.obj
 0002:00002dac       ??_C@_03IKGEINEE@?$CFs?5@  1001bdac     hprof_io.obj
 0002:00002db0       ??_C@_0BB@CNGBILFI@?$DMunknown?5caller?$DO@ 1001bdb0     hprof_io.obj
 0002:00002dc4       ??_C@_03PMGGPEJJ@?$CFd?6@  1001bdc4     hprof_io.obj
 0002:00002dc8       ??_C@_0CG@OEAEBDMP@MONITOR?5TIME?5BEGIN?5?$CItotal?5?$DN?5?$CFu?5@ 1001bdc8     hprof_io.obj
 0002:00002df0       ??_C@_0CK@EIFBODMG@rank?5?5?5self?5?5accum?5?5?5count?5trac@ 1001bdf0     hprof_io.obj
 0002:00002e1c       ??_C@_0CH@DCKBGDHE@?$CF4u?5?$CF5?42f?$CF?$CF?5?$CF5?42f?$CF?$CF?5?$CF7u?5?$CF5u?5?$CFs?5@ 1001be1c     hprof_io.obj
 0002:00002e44       ??_C@_0BC@NJINABM@MONITOR?5TIME?5END?6@ 1001be44     hprof_io.obj
 0002:00002e58       ??_C@_0CF@GOKDFEGE@SLEEP?3?5timeout?$DN?$CFd?0?5?$DMunknown?5thr@ 1001be58     hprof_io.obj
 0002:00002e80       ??_C@_0BO@BIEEFEKH@SLEEP?3?5timeout?$DN?$CFd?0?5thread?5?$CFd?6@ 1001be80     hprof_io.obj
 0002:00002ea0       ??_C@_0DA@PAOIGCJK@WAIT?3?5MONITOR?5?$CFs?0?5timeout?$DN?$CFd?0?5?$DM@ 1001bea0     hprof_io.obj
 0002:00002ed0       ??_C@_0CJ@JDGFDGCO@WAIT?3?5MONITOR?5?$CFs?0?5timeout?$DN?$CFd?0?5t@ 1001bed0     hprof_io.obj
 0002:00002efc       ??_C@_0DG@JKNMLIIB@WAITED?3?5MONITOR?5?$CFs?0?5time_waited@ 1001befc     hprof_io.obj
 0002:00002f34       ??_C@_0CP@KECIBELF@WAITED?3?5MONITOR?5?$CFs?0?5time_waited@ 1001bf34     hprof_io.obj
 0002:00002f64       ??_C@_0BE@MPINDFNB@MONITOR?5DUMP?5BEGIN?6@ 1001bf64     hprof_io.obj
 0002:00002f78       ??_C@_02ONMOIAPO@S?$HM@    1001bf78     hprof_io.obj
 0002:00002f7c       ??_C@_05HHGGHEON@intr?$HM@ 1001bf7c     hprof_io.obj
 0002:00002f84       ??_C@_07PFCOEPNE@native?$HM@ 1001bf84     hprof_io.obj
 0002:00002f8c       ??_C@_02BGHENOEB@ZO@       1001bf8c     hprof_io.obj
 0002:00002f90       ??_C@_02OLCMIILA@NS@       1001bf90     hprof_io.obj
 0002:00002f94       ??_C@_02DCIILGAN@SL@       1001bf94     hprof_io.obj
 0002:00002f98       ??_C@_02INAGPDON@MW@       1001bf98     hprof_io.obj
 0002:00002f9c       ??_C@_02IHJINOOH@CW@       1001bf9c     hprof_io.obj
 0002:00002fa0       ??_C@_01DGKLNCNG@R@        1001bfa0     hprof_io.obj
 0002:00002fa4       ??_C@_02EDDKIDN@UN@        1001bfa4     hprof_io.obj
 0002:00002fa8       ??_C@_0CF@EEKKPGCA@?5?5?5?5THREAD?5?$CFd?0?5trace?5?$CFd?0?5status@ 1001bfa8     hprof_io.obj
 0002:00002fd0       ??_C@_0BA@DDIGAEMH@?5?5?5?5MONITOR?5?$CFs?6@ 1001bfd0     hprof_io.obj
 0002:00002fe0       ??_C@_0CE@GMJCPGJB@?7owner?3?5thread?5?$CFd?0?5entry?5count?3@ 1001bfe0     hprof_io.obj
 0002:00003004       ??_C@_0BI@HJHMLMLK@?5?5?5?5MONITOR?5?$CFs?5unowned?6@ 1001c004     hprof_io.obj
 0002:0000301c       ??_C@_0BD@FPGLBOLN@?7waiting?5to?5enter?3@ 1001c01c     hprof_io.obj
 0002:00003030       ??_C@_0BJ@JNJDPIMA@?7waiting?5to?5be?5notified?3@ 1001c030     hprof_io.obj
 0002:0000304c       ??_C@_0BC@FFCEFDPI@MONITOR?5DUMP?5END?6@ 1001c04c     hprof_io.obj
 0002:00003060       ??_C@_0CK@EJNNGPCB@HEAP?5DUMP?5BEGIN?5?$CI?$CFu?5objects?0?5?$CFu@ 1001c060     hprof_io.obj
 0002:0000308c       ??_C@_0CK@NFEGAEJI@ROOT?5?$CFx?5?$CIkind?$DN?$DMthread?$DO?0?5id?$DN?$CFu?0?5@ 1001c08c     hprof_io.obj
 0002:000030b8       ??_C@_0BK@JNDLAOIB@ROOT?5?$CFx?5?$CIkind?$DN?$DMunknown?$DO?$CJ?6@ 1001c0b8     hprof_io.obj
 0002:000030d4       ??_C@_0DC@MOCOIGOI@ROOT?5?$CFx?5?$CIkind?$DN?$DMJNI?5global?5ref?$DO?0@ 1001c0d4     hprof_io.obj
 0002:00003108       ??_C@_0DF@EHNMLMKL@ROOT?5?$CFx?5?$CIkind?$DN?$DMJNI?5local?5ref?$DO?0?5@ 1001c108     hprof_io.obj
 0002:00003140       ??_C@_0CI@HPDPNKKD@ROOT?5?$CFx?5?$CIkind?$DN?$DMsystem?5class?$DO?0?5n@ 1001c140     hprof_io.obj
 0002:00003168       ??_C@_0BP@DMJMIOPP@ROOT?5?$CFx?5?$CIkind?$DN?$DMbusy?5monitor?$DO?$CJ?6@ 1001c168     hprof_io.obj
 0002:00003188       ??_C@_0CK@NCNELCJJ@ROOT?5?$CFx?5?$CIkind?$DN?$DMthread?5block?$DO?0?5t@ 1001c188     hprof_io.obj
 0002:000031b4       ??_C@_0DC@GMGLBKOF@ROOT?5?$CFx?5?$CIkind?$DN?$DMJava?5stack?$DO?0?5thr@ 1001c1b4     hprof_io.obj
 0002:000031e8       ??_C@_0CJ@BBCGEJMI@Mis?9match?5on?5instance?5size?5in?5c@ 1001c1e8     hprof_io.obj
 0002:00003214       ??_C@_0BM@LKLLFLPM@CLS?5?$CFx?5?$CIname?$DN?$CFs?0?5trace?$DN?$CFu?$CJ?6@ 1001c214     hprof_io.obj
 0002:00003230       ??_C@_0M@GAICGIPA@?7super?7?7?$CFx?6@ 1001c230     hprof_io.obj
 0002:0000323c       ??_C@_0N@FIMCJNAO@?7loader?7?7?$CFx?6@ 1001c23c     hprof_io.obj
 0002:0000324c       ??_C@_0O@LMOJKNLE@?7signers?7?7?$CFx?6@ 1001c24c     hprof_io.obj
 0002:0000325c       ??_C@_0N@PJLEKNME@?7domain?7?7?$CFx?6@ 1001c25c     hprof_io.obj
 0002:0000326c       ??_C@_0P@NELJBPCL@?7static?5?$CFs?7?$CFx?6@ 1001c26c     hprof_io.obj
 0002:0000327c       ??_C@_0BM@BBCDPNOI@?7constant?5pool?5entry?5?$CFd?7?$CFx?6@ 1001c27c     hprof_io.obj
 0002:00003298       ??_C@_0CM@FKBOPKCE@Mis?9match?5on?5instance?5size?5in?5i@ 1001c298     hprof_io.obj
 0002:000032c4       ??_C@_0CH@PDBDJJN@OBJ?5?$CFx?5?$CIsz?$DN?$CFu?0?5trace?$DN?$CFu?0?5class?$DN@ 1001c2c4     hprof_io.obj
 0002:000032ec       ??_C@_01GPOEFGEJ@?7@       1001c2ec     hprof_io.obj
 0002:000032f0       ??_C@_09EBLDCIPL@?7?$CFs?7?$CFs?$CFx?6@ 1001c2f0     hprof_io.obj
 0002:000032fc       ??_C@_0DG@OEIOANKC@ARR?5?$CFx?5?$CIsz?$DN?$CFu?0?5trace?$DN?$CFu?0?5nelems@ 1001c2fc     hprof_io.obj
 0002:00003334       ??_C@_0L@NNOLGAJB@?7?$FL?$CFu?$FN?7?7?$CFx?6@ 1001c334     hprof_io.obj
 0002:00003340       ??_C@_0DD@KCKFMPAB@ARR?5?$CFx?5?$CIsz?$DN?$CFu?0?5trace?$DN?$CFu?0?5nelems@ 1001c340     hprof_io.obj
 0002:00003374       ??_C@_0CI@FAOICMFN@File?5size?5is?5smaller?5than?5bytes@ 1001c374     hprof_io.obj
 0002:0000339c       ??_C@_0CL@FLNKDKBO@Cannot?5seek?5to?5beginning?5of?5hea@ 1001c39c     hprof_io.obj
 0002:000033c8       ??_C@_0P@GNGJOCHE@HEAP?5DUMP?5END?6@ 1001c3c8     hprof_io.obj
 0002:000033d8       __real@4059000000000000    1001c3d8     hprof_io.obj
 0002:000033e0       ??_C@_07MDLDPMJN@IoNames@  1001c3e0     hprof_ioname.obj
 0002:000033e8       ??_C@_0CJ@HGLEALFG@HPROF?3?5received?5exit?5event?0?5exi@ 1001c3e8     hprof_listener.obj
 0002:00003414       ??_C@_0CG@FEEGFMIO@failed?5to?5recognize?5cmd?5?$CFd?0?5exi@ 1001c414     hprof_listener.obj
 0002:0000343c       ??_C@_0BB@HJHGLACE@hprof_listener?4c@ 1001c43c     hprof_listener.obj
 0002:00003450       ??_C@_0BE@HPBGIMIM@HPROF?5listener?5lock@ 1001c450     hprof_listener.obj
 0002:00003464       ??_C@_0BG@MPNHEDPO@HPROF?5listener?5thread@ 1001c464     hprof_listener.obj
 0002:0000347c       ??_C@_0CO@FNPLHOCK@Loader?50x?$CF08x?3?5globalref?$DN?$CFp?0?5ob@ 1001c47c     hprof_loader.obj
 0002:000034ac       ??_C@_06FLJJKOBF@Loader@   1001c4ac     hprof_loader.obj
 0002:000034b4       ??_C@_0DN@EAGMNPFH@?9?9?9?9?9?9?9?9?9?9?9?9?9?9?9?9?9?9?9?9?9?5Loader?5Ta@ 1001c4b4     hprof_loader.obj
 0002:000034f4       ??_C@_09EFPGAEIO@?$CFs?2lib?2?$CFs@ 1001c4f4     hprof_md.obj
 0002:00003500       ??_C@_01ICJEACDI@?$DL@     1001c500     hprof_md.obj
 0002:00003504       ??_C@_09CMKFMIAO@?$CFs?2?$CFs?4dll@ 1001c504     hprof_md.obj
 0002:00003510       ??_C@_06DAJAKOAL@?$CFs?4dll@ 1001c510     hprof_md.obj
 0002:00003518       ??_C@_0BP@KMBPCJLM@Can?8t?5find?5dependent?5libraries@ 1001c518     hprof_md.obj
 0002:00003538       ??_C@_0EP@IMBLBEBH@Monitor?50x?$CF08x?3?5trace?$DN0x?$CF08x?0?5s@ 1001c538     hprof_monitor.obj
 0002:00003588       ??_C@_07EJLIBABC@Monitor@  1001c588     hprof_monitor.obj
 0002:00003590       ??_C@_0DM@CDMHECPA@?9?9?9?9?9?9?9?9?9?9?9?9?9?9?9?9?9?9?9?5Monitor?5Tab@ 1001c590     hprof_monitor.obj
 0002:000035d0       ??_C@_0EO@FJDPGHOM@Object?50x?$CF08x?3?5site?$DN0x?$CF08x?0?5SN?$DN@ 1001c5d0     hprof_object.obj
 0002:00003620       ??_C@_06ELFECKBG@Object@   1001c620     hprof_object.obj
 0002:00003628       ??_C@_0DN@PGMDODNP@?9?9?9?9?9?9?9?9?9?9?9?9?9?9?9?9?9?9?9?9?9?5Object?5Ta@ 1001c628     hprof_object.obj
 0002:00003668       ??_C@_0FD@PFDMHJMO@?$FL?$CFd?$FN?3?5flavor?$DN?$CFd?0?5refKind?$DN?$CFd?0?5pr@ 1001c668     hprof_reference.obj
 0002:000036bc       ??_C@_0BO@HLFIJNLO@?6FOLLOW?5REFERENCES?5RETURNED?3?6@ 1001c6bc     hprof_reference.obj
 0002:000036dc       ??_C@_0BC@CBPNKGLB@?$FL?$CFd?$FN?5?$CFs?5?$CC?$CFs?$CC?5?$CC?$CFs?$CC@ 1001c6dc     hprof_reference.obj
 0002:000036f0       ??_C@_0BC@DFPEGHHN@?5?$CIprimType?$DN?$CFd?$CI?$CFc?$CJ@ 1001c6f0     hprof_reference.obj
 0002:00003704       ??_C@_0N@KKCODGGO@?0?5got?5?$CFd?$CI?$CFc?$CJ@ 1001c704     hprof_reference.obj
 0002:00003714       ??_C@_01PKGAHCOL@?$CJ@     1001c714     hprof_reference.obj
 0002:00003718       ??_C@_08BLCEBNNI@?$CIty?$DNOBJ?$CJ@ 1001c718     hprof_reference.obj
 0002:00003724       ??_C@_0CI@MODAHCDH@?5val?$DN?$FL0x?$CF08x?00x?$CF08x?$FN?5or?5?$FL0x?$CF08x@ 1001c724     hprof_reference.obj
 0002:0000374c       ??_C@_0BM@PKNIEFFF@?6HPROF?5LIST?5OF?5ALL?5FIELDS?3?6@ 1001c74c     hprof_reference.obj
 0002:00003768       ??_C@_0BA@BFMBFEDH@?6PROBLEM?5WITH?3?6@ 1001c768     hprof_reference.obj
 0002:00003778       ??_C@_0BC@JAMMPJCI@hprof_reference?4c@ 1001c778     hprof_reference.obj
 0002:0000378c       ??_C@_0CC@KOEPIMAA@Trouble?5with?5fields?5and?5heap?5da@ 1001c78c     hprof_reference.obj
 0002:000037b0       ??_C@_0CG@LOGJKIDP@Unprepared?5class?5with?5reference@ 1001c7b0     hprof_reference.obj
 0002:000037d8       ??_C@_0CA@HDCNGDOI@Trouble?5with?5unprepared?5classes@ 1001c7d8     hprof_reference.obj
 0002:000037f8       ??_C@_0CM@KOJHGKPG@Instance?5of?5unprepared?5class?5wi@ 1001c7f8     hprof_reference.obj
 0002:00003824       ??_C@_0CP@PGGCECJG@Instance?5of?5unprepared?5class?5wi@ 1001c824     hprof_reference.obj
 0002:00003854       ??_C@_0CM@LCFNMMIH@Big?5Trouble?5with?5unprepared?5cla@ 1001c854     hprof_reference.obj
 0002:00003880       ??_C@_03MCAECCCA@Ref@      1001c880     hprof_reference.obj
 0002:00003888       ??_C@_0GL@CKPFBEEL@Site?50x?$CF08x?3?5class?$DN0x?$CF08x?0?5trac@ 1001c888     hprof_site.obj
 0002:000038f4       ??_C@_04ELDCFKBO@Site@     1001c8f4     hprof_site.obj
 0002:000038fc       ??_C@_0DL@GINFEJKL@?9?9?9?9?9?9?9?9?9?9?9?9?9?9?9?9?9?9?9?9?9?5Site?5Tabl@ 1001c8fc     hprof_site.obj
 0002:00003938       ??_C@_0BA@KPHMOMNK@allocated?5bytes@ 1001c938     hprof_site.obj
 0002:00003948       ??_C@_0L@CIOGHAJA@live?5bytes@ 1001c948     hprof_site.obj
 0002:00003954       ??_C@_07NBCGADJA@Unknown@  1001c954     hprof_site.obj
 0002:00003960       __xmm@41f00000000000000000000000000000 1001c960     hprof_site.obj
 0002:00003970       ??_C@_07BJOIOONN@Strings@  1001c970     hprof_string.obj
 0002:00003978       ??_C@_0BF@CMBFGNJH@0x?$CF08x?3?5String?5?$CC?$CFs?$CC?6@ 1001c978     hprof_string.obj
 0002:00003990       ??_C@_0DM@EIBMKCIH@?9?9?9?9?9?9?9?9?9?9?9?9?9?9?9?9?9?9?9?9?5String?5Tab@ 1001c990     hprof_string.obj
 0002:000039cc       ??_C@_0O@DNKFFEDP@hprof_table?4c@ 1001c9cc     hprof_table.obj
 0002:000039dc       ??_C@_0CI@BKFDBKDO@SANITY?5IN?5QUESTION?3?5new_size?5?$DO?5@ 1001c9dc     hprof_table.obj
 0002:00003a04       ??_C@_0BE@HKNCGDI@HPROF?5?$CFs?5table?5lock@ 1001ca04     hprof_table.obj
 0002:00003a18       ??_C@_0EB@ECOEHIOB@SANITY?5IN?5QUESTION?3?5SANITY_ADD_@ 1001ca18     hprof_table.obj
 0002:00003a5c       ??_C@_0DB@BICPHHBL@SANITY?5IN?5QUESTION?3?5?$CIindex?$CJ?5?$DM?5l@ 1001ca5c     hprof_table.obj
 0002:00003a90       ??_C@_0M@IDKNHDJ@hprof_tag?4c@ 1001ca90     hprof_tag.obj
 0002:00003a9c       ??_C@_0CP@CMIJBALN@JVMTI?5tag?5value?5is?5not?50?5and?5mi@ 1001ca9c     hprof_tag.obj
 0002:00003ad0       ??_C@_0FN@BEJBEIPH@Tls?50x?$CF08x?3?5SN?$DN?$CFu?0?5sample_statu@ 1001cad0     hprof_tls.obj
 0002:00003b30       ??_C@_0M@CPNBNDEA@hprof_tls?4c@ 1001cb30     hprof_tls.obj
 0002:00003b3c       ??_C@_0CE@FEDDBDEF@no?5frames?0?5method?5can?8t?5be?5on?5s@ 1001cb3c     hprof_tls.obj
 0002:00003b60       ??_C@_0CK@PCBPHOKB@method?5return?5tracked?0?5but?5stac@ 1001cb60     hprof_tls.obj
 0002:00003b8c       ??_C@_03HCMCMCCF@TLS@      1001cb8c     hprof_tls.obj
 0002:00003b90       ??_C@_0DK@IDPJJJOO@?9?9?9?9?9?9?9?9?9?9?9?9?9?9?9?9?9?9?9?9?9?5TLS?5Table@ 1001cb90     hprof_tls.obj
 0002:00003bcc       ??_C@_0CA@GKPNPPJP@expection?5pop?0?5nothing?5on?5stack@ 1001cbcc     hprof_tls.obj
 0002:00003bec       ??_C@_0BK@CANKCPKH@exception?5pop?5stack?5empty@ 1001cbec     hprof_tls.obj
 0002:00003c08       ??_C@_0DI@GKCOFGK@Trace?50x?$CF08x?3?5SN?$DN?$CFu?0?5threadSN?$DN?$CF@ 1001cc08     hprof_trace.obj
 0002:00003c40       ??_C@_08EKIEFACC@0x?$CF08x?0?5@ 1001cc40     hprof_trace.obj
 0002:00003c50       ??_C@_0FC@DNOAGMNM@?$CJ?0?5traceSN?$DN?$CFu?0?5num_hits?$DN?$CFd?0?5sel@ 1001cc50     hprof_trace.obj
 0002:00003ca4       ??_C@_05ILLBNNOP@Trace@    1001cca4     hprof_trace.obj
 0002:00003cac       ??_C@_0DM@MBLFMP@?9?9?9?9?9?9?9?9?9?9?9?9?9?9?9?9?9?9?9?9?9?5Trace?5Tab@ 1001ccac     hprof_trace.obj
 0002:00003ce8       ??_C@_0P@OOAACBOI@nativeNewArray@ 1001cce8     hprof_tracker.obj
 0002:00003cf8       ??_C@_0CI@PCHNGLLD@?$CILjava?1lang?1Object?$DLLjava?1lang?1O@ 1001ccf8     hprof_tracker.obj
 0002:00003d20       ??_C@_0BB@POPFLJFA@nativeObjectInit@ 1001cd20     hprof_tracker.obj
 0002:00003d34       ??_C@_0P@MCMNPMHF@nativeCallSite@ 1001cd34     hprof_tracker.obj
 0002:00003d44       ??_C@_0BI@HJMIOFJM@?$CILjava?1lang?1Object?$DLII?$CJV@ 1001cd44     hprof_tracker.obj
 0002:00003d5c       ??_C@_0BB@PCLGJBAD@nativeReturnSite@ 1001cd5c     hprof_tracker.obj
 0002:00003d70       ??_C@_0BA@FINNOAJG@hprof_tracker?4c@ 1001cd70     hprof_tracker.obj
 0002:00003d80       ??_C@_0BM@NEBJJKBP@Problems?5tracking?5callbacks@ 1001cd80     hprof_tracker.obj
 0002:00003d9c       ??_C@_01JPJNBJEM@I@        1001cd9c     hprof_tracker.obj
 0002:00003da0       ??_C@_07IBIALADM@engaged@  1001cda0     hprof_tracker.obj
 0002:00003da8       ??_C@_0CG@CBMHIAIE@Unexpected?5Exception?5found?5befo@ 1001cda8     hprof_tracker.obj
 0002:00003dd0       ??_C@_0CF@PCFIAEGA@Unexpected?5Exception?5found?5afte@ 1001cdd0     hprof_tracker.obj
 0002:00003df8       ??_C@_03GAEACAIP@?$CI?$CJV@ 1001cdf8     hprof_tracker.obj
 0002:00003dfc       ??_C@_06FALKBLGB@?$DMinit?$DO@ 1001cdfc     hprof_tracker.obj
 0002:00003e08       ??_C@_0GL@KMNNLEBA@Unable?5to?5access?5JNI?5Version?51?4@ 1001ce08     hprof_util.obj
 0002:00003e74       ??_C@_0N@BCNOCCGD@hprof_util?4c@ 1001ce74     hprof_util.obj
 0002:00003e84       ??_C@_0BN@JBCFKHE@Cannot?5allocate?5jvmti?5memory@ 1001ce84     hprof_util.obj
 0002:00003ea4       ??_C@_0BP@MLLANJPH@Cannot?5deallocate?5jvmti?5memory@ 1001cea4     hprof_util.obj
 0002:00003ec4       ??_C@_0BO@NJHGGBBD@Cannot?5allocate?5malloc?5memory@ 1001cec4     hprof_util.obj
 0002:00003ee4       ??_C@_0CA@JOBIPEPH@Cannot?5get?5jvmti?5version?5number@ 1001cee4     hprof_util.obj
 0002:00003f04       ??_C@_0BK@OAILAOGO@Cannot?5create?5raw?5monitor@ 1001cf04     hprof_util.obj
 0002:00003f20       ??_C@_0BO@HMGKMEHC@Cannot?5enter?5with?5raw?5monitor@ 1001cf20     hprof_util.obj
 0002:00003f40       ??_C@_0BN@LFBKBPAF@Cannot?5wait?5with?5raw?5monitor@ 1001cf40     hprof_util.obj
 0002:00003f60       ??_C@_0CD@GFHMPPID@Cannot?5notify?5all?5with?5raw?5moni@ 1001cf60     hprof_util.obj
 0002:00003f84       ??_C@_0BN@MDHBAEMA@Cannot?5exit?5with?5raw?5monitor@ 1001cf84     hprof_util.obj
 0002:00003fa4       ??_C@_0BL@KDPPDKJE@Cannot?5destroy?5raw?5monitor@ 1001cfa4     hprof_util.obj
 0002:00003fc0       ??_C@_0BO@HBJLHGJI@Cannot?5set?5event?5notification@ 1001cfc0     hprof_util.obj
 0002:00003fe0       ??_C@_0CF@ODOPAONB@JNI?5PushLocalFrame?5returned?5non@ 1001cfe0     hprof_util.obj
 0002:00004008       ??_C@_0CI@GNJHOCCG@JNI?5PopLocalFrame?5returned?5wron@ 1001d008     hprof_util.obj
 0002:00004030       ??_C@_0CG@INKKJECJ@JNI?5RegisterNatives?5returned?5no@ 1001d030     hprof_util.obj
 0002:00004058       ??_C@_06FKJAAAAK@onload@   1001d058     hprof_util.obj
 0002:00004060       ??_C@_0L@LCBNLHKO@primordial@ 1001d060     hprof_util.obj
 0002:0000406c       ??_C@_05FAGFPHJG@start@    1001d06c     hprof_util.obj
 0002:00004074       ??_C@_04GLMHKBCH@live@     1001d074     hprof_util.obj
 0002:0000407c       ??_C@_04BBBDNBOK@dead@     1001d07c     hprof_util.obj
 0002:00004084       ??_C@_07CIFAGBMG@unknown@  1001d084     hprof_util.obj
 0002:0000408c       ??_C@_0BH@GGEPPPJA@Cannot?5get?5object?5size@ 1001d08c     hprof_util.obj
 0002:000040a4       ??_C@_0BI@PBBMGKKM@Cannot?5call?5IsInterface@ 1001d0a4     hprof_util.obj
 0002:000040bc       ??_C@_0BI@DAHMAJNN@Cannot?5get?5class?5status@ 1001d0bc     hprof_util.obj
 0002:000040d4       ??_C@_0BI@JNNPNCAM@Cannot?5get?5class?5loader@ 1001d0d4     hprof_util.obj
 0002:000040ec       ??_C@_0BG@BILEMKBA@Cannot?5get?5object?5tag@ 1001d0ec     hprof_util.obj
 0002:00004104       ??_C@_0BG@NGKKDADM@Cannot?5set?5object?5tag@ 1001d104     hprof_util.obj
 0002:0000411c       ??_C@_0BO@KIPAKMFC@Cannot?5get?5monitor?5usage?5info@ 1001d11c     hprof_util.obj
 0002:0000413c       ??_C@_0CF@PLCCHECM@Cannot?5get?5thread?5owned?5monitor@ 1001d13c     hprof_util.obj
 0002:00004164       ??_C@_0BL@NDMINGDE@Cannot?5get?5system?5property@ 1001d164     hprof_util.obj
 0002:00004180       ??_C@_0BL@GMBHKAMD@Cannot?5get?5class?5signature@ 1001d180     hprof_util.obj
 0002:0000419c       ??_C@_0BM@MJKLBGEI@Cannot?5get?5source?5file?5name@ 1001d19c     hprof_util.obj
 0002:000041b8       ??_C@_0CH@KOOPIIML@Class?5not?5prepared?5when?5needing@ 1001d1b8     hprof_util.obj
 0002:000041e0       ??_C@_0BM@MNEEOAMD@Cannot?5get?5class?5field?5list@ 1001d1e0     hprof_util.obj
 0002:000041fc       ??_C@_0BL@BPDDELKG@Cannot?5get?5field?5modifiers@ 1001d1fc     hprof_util.obj
 0002:00004218       ??_C@_0BG@LCHPHFJE@Cannot?5get?5field?5name@ 1001d218     hprof_util.obj
 0002:00004230       ??_C@_0CA@FINGKAAM@Cannot?5get?5class?5interface?5list@ 1001d230     hprof_util.obj
 0002:00004250       ??_C@_0BI@LGAMFNKM@Class?5signature?5is?3?5?$CFs?6@ 1001d250     hprof_util.obj
 0002:00004268       ??_C@_0CL@OFFNDEFG@Class?5not?5prepared?5when?5needing@ 1001d268     hprof_util.obj
 0002:00004294       ??_C@_0BI@CHMLIOLP@Cannot?5get?5method?5class@ 1001d294     hprof_util.obj
 0002:000042ac       ??_C@_0BO@PAPBMIBC@Cannot?5check?5is?5method?5native@ 1001d2ac     hprof_util.obj
 0002:000042cc       ??_C@_0BH@BPLLGFCI@Cannot?5get?5method?5name@ 1001d2cc     hprof_util.obj
 0002:000042e4       ??_C@_0CM@GKGAKFLL@Unable?5to?5get?5potential?5JVMTI?5c@ 1001d2e4     hprof_util.obj
 0002:00004310       ??_C@_0CM@GHHLBMIK@Unable?5to?5get?5necessary?5JVMTI?5c@ 1001d310     hprof_util.obj
 0002:0000433c       ??_C@_0BL@IPIJPPGI@Cannot?5set?5jvmti?5callbacks@ 1001d33c     hprof_util.obj
 0002:00004358       ??_C@_0CA@IEJEDHCB@Cannot?5get?5thread?5local?5storage@ 1001d358     hprof_util.obj
 0002:00004378       ??_C@_0CA@CHDOFKLE@Cannot?5set?5thread?5local?5storage@ 1001d378     hprof_util.obj
 0002:00004398       ??_C@_0BI@BFOOMEII@Cannot?5get?5thread?5state@ 1001d398     hprof_util.obj
 0002:000043b0       ??_C@_0BH@LALMLBEN@Cannot?5get?5thread?5info@ 1001d3b0     hprof_util.obj
 0002:000043c8       ??_C@_0BN@CIIHGGBH@Cannot?5get?5thread?5group?5info@ 1001d3c8     hprof_util.obj
 0002:000043e8       ??_C@_0CB@OOIBEDA@Cannot?5get?5all?5loaded?5class?5lis@ 1001d3e8     hprof_util.obj
 0002:0000440c       ??_C@_0BP@DPAIDJBG@Cannot?5get?5source?5line?5numbers@ 1001d40c     hprof_util.obj
 0002:0000442c       ??_C@_0BC@LHBANJHF@java?1lang?1Runtime@ 1001d42c     hprof_util.obj
 0002:00004440       ??_C@_0BG@JELJIEND@?$CI?$CJLjava?1lang?1Runtime?$DL@ 1001d440     hprof_util.obj
 0002:00004458       ??_C@_0L@POECMMEP@getRuntime@ 1001d458     hprof_util.obj
 0002:00004464       ??_C@_03IGDHHNNC@?$CI?$CJJ@ 1001d464     hprof_util.obj
 0002:00004468       ??_C@_09NKELKHPD@maxMemory@ 1001d468     hprof_util.obj
 0002:00004474       ??_C@_0CN@EFABAIOP@?$CILjava?1lang?1ThreadGroup?$DLLjava?1l@ 1001d474     hprof_util.obj
 0002:000044a4       ??_C@_04LHKBAEFM@?$CIZ?$CJV@ 1001d4a4     hprof_util.obj
 0002:000044ac       ??_C@_09GMGCGCNB@setDaemon@ 1001d4ac     hprof_util.obj
 0002:000044b8       ??_C@_0BL@DNNDHALM@Cannot?5create?5agent?5thread@ 1001d4b8     hprof_util.obj
 0002:000044d4       ??_C@_0CC@KOBPHIDN@Cannot?5get?5thread?5list?5stack?5in@ 1001d4d4     hprof_util.obj
 0002:000044f8       ??_C@_0BJ@KKFDNCKO@Cannot?5follow?5references@ 1001d4f8     hprof_util.obj
 0002:00004514       ??_C@_0CA@HHGMNCL@Cannot?5force?5garbage?5collection@ 1001d514     hprof_util.obj
 0002:00004538       ??_C@_0GL@PEBNFMGB@Unable?5to?5access?5JVMTI?5Version?5@ 1001d538     hprof_util.obj
 0002:000045a8       ??_C@_0GP@FALDBDHK@This?5hprof?5native?5library?5will?5@ 1001d5a8     hprof_util.obj
 0002:00004638       __pDefaultRawDllMain       1001d638     MSVCRT:dll_dllmain.obj
 0002:00004638       __pRawDllMain              1001d638     MSVCRT:dll_dllmain.obj
 0002:00004648       __load_config_used         1001d648     MSVCRT:loadcfg.obj
 0002:00004780       ___safe_se_handler_table   1001d780     <linker-defined>
 0002:00004784       ___volatile_metadata       1001d784     <linker-defined>
 0002:00004b48       ___rtc_iaa                 1001db48     MSVCRT:initsect.obj
 0002:00004b4c       ___rtc_izz                 1001db4c     MSVCRT:initsect.obj
 0002:00004b50       ___rtc_taa                 1001db50     MSVCRT:initsect.obj
 0002:00004b54       ___rtc_tzz                 1001db54     MSVCRT:initsect.obj
 0002:00004c4c       __IMPORT_DESCRIPTOR_WSOCK32 1001dc4c     wsock32:WSOCK32.dll
 0002:00004c60       __IMPORT_DESCRIPTOR_WINMM  1001dc60     winmm:WINMM.dll
 0002:00004c74       __IMPORT_DESCRIPTOR_KERNEL32 1001dc74     kernel32:KERNEL32.dll
 0002:00004c88       __IMPORT_DESCRIPTOR_VCRUNTIME140 1001dc88     vcruntime:VCRUNTIME140.dll
 0002:00004c9c       __IMPORT_DESCRIPTOR_api-ms-win-crt-runtime-l1-1-0 1001dc9c     ucrt:api-ms-win-crt-runtime-l1-1-0.dll
 0002:00004cb0       __IMPORT_DESCRIPTOR_api-ms-win-crt-string-l1-1-0 1001dcb0     ucrt:api-ms-win-crt-string-l1-1-0.dll
 0002:00004cc4       __IMPORT_DESCRIPTOR_api-ms-win-crt-stdio-l1-1-0 1001dcc4     ucrt:api-ms-win-crt-stdio-l1-1-0.dll
 0002:00004cd8       __IMPORT_DESCRIPTOR_api-ms-win-crt-filesystem-l1-1-0 1001dcd8     ucrt:api-ms-win-crt-filesystem-l1-1-0.dll
 0002:00004cec       __IMPORT_DESCRIPTOR_api-ms-win-crt-heap-l1-1-0 1001dcec     ucrt:api-ms-win-crt-heap-l1-1-0.dll
 0002:00004d00       __IMPORT_DESCRIPTOR_api-ms-win-crt-convert-l1-1-0 1001dd00     ucrt:api-ms-win-crt-convert-l1-1-0.dll
 0002:00004d14       __IMPORT_DESCRIPTOR_api-ms-win-crt-environment-l1-1-0 1001dd14     ucrt:api-ms-win-crt-environment-l1-1-0.dll
 0002:00004d28       __IMPORT_DESCRIPTOR_api-ms-win-crt-time-l1-1-0 1001dd28     ucrt:api-ms-win-crt-time-l1-1-0.dll
 0002:00004d3c       __IMPORT_DESCRIPTOR_api-ms-win-crt-utility-l1-1-0 1001dd3c     ucrt:api-ms-win-crt-utility-l1-1-0.dll
 0002:00004d50       __NULL_IMPORT_DESCRIPTOR   1001dd50     wsock32:WSOCK32.dll
 0003:00000108       ___security_cookie_complement 1001f108     MSVCRT:gs_cookie.obj
 0003:0000010c       ___security_cookie         1001f10c     MSVCRT:gs_cookie.obj
 0003:00000110       __fltused                  1001f110     MSVCRT:fltused.obj
 0003:00000120       ___isa_enabled             1001f120     MSVCRT:cpu_disp.obj
 0003:00000124       ___scrt_native_dllmain_reason 1001f124     MSVCRT:utility.obj
 0003:00000130       ___scrt_ucrt_dll_is_in_use 1001f130     MSVCRT:ucrt_stubs.obj
 0003:000007ec       ___isa_available           1001f7ec     MSVCRT:cpu_disp.obj
 0003:000007f0       ___favor                   1001f7f0     MSVCRT:cpu_disp.obj
 0003:000007f8       ?__type_info_root_node@@3U__type_info_node@@A 1001f7f8     MSVCRT:tncleanup.obj
 0003:00000800       ?_OptionsStorage@?1??__local_stdio_scanf_options@@9@4_KA 1001f800     MSVCRT:default_local_stdio_options.obj
 0003:00000808       ___scrt_current_native_startup_state 1001f808     MSVCRT:utility.obj
 0003:0000080c       ___scrt_native_startup_lock 1001f80c     MSVCRT:utility.obj
 0003:0000082c       ___scrt_debugger_hook_flag 1001f82c     MSVCRT:utility_desktop.obj
 0003:00000830       _hJavaInst                 1001f830     <common>
 0003:00000834       _gdata                     1001f834     <common>
 0003:00000838       ?_OptionsStorage@?1??__local_stdio_printf_options@@9@9 1001f838     <common>
 0003:00000840       ___dyn_tls_init_callback   1001f840     <common>

 entry point at        0001:000174e1

 Static symbols

 0000:fffdd000       .debug$S                   10000000     hprof.exp
 0000:fffdd000       .debug$S                   10000000     vcruntime:VCRUNTIME140.dll
 0000:fffdd000       .debug$S                   10000000     vcruntime:VCRUNTIME140.dll
 0000:fffdd000       .debug$S                   10000000     vcruntime:VCRUNTIME140.dll
 0000:fffdd000       .debug$S                   10000000     vcruntime:VCRUNTIME140.dll
 0000:fffdd000       .debug$S                   10000000     vcruntime:VCRUNTIME140.dll
 0000:fffdd000       .debug$S                   10000000     vcruntime:VCRUNTIME140.dll
 0000:fffdd000       .debug$S                   10000000     vcruntime:VCRUNTIME140.dll
 0000:fffdd000       .debug$S                   10000000     vcruntime:VCRUNTIME140.dll
 0000:fffdd000       .debug$S                   10000000     ucrt:api-ms-win-crt-convert-l1-1-0.dll
 0000:fffdd000       .debug$S                   10000000     ucrt:api-ms-win-crt-convert-l1-1-0.dll
 0000:fffdd000       .debug$S                   10000000     ucrt:api-ms-win-crt-environment-l1-1-0.dll
 0000:fffdd000       .debug$S                   10000000     ucrt:api-ms-win-crt-filesystem-l1-1-0.dll
 0000:fffdd000       .debug$S                   10000000     ucrt:api-ms-win-crt-filesystem-l1-1-0.dll
 0000:fffdd000       .debug$S                   10000000     ucrt:api-ms-win-crt-heap-l1-1-0.dll
 0000:fffdd000       .debug$S                   10000000     ucrt:api-ms-win-crt-heap-l1-1-0.dll
 0000:fffdd000       .debug$S                   10000000     ucrt:api-ms-win-crt-math-l1-1-0.dll
 0002:fffe7000       .idata$6                   10000000     ucrt:api-ms-win-crt-math-l1-1-0.dll
 0000:fffdd000       .debug$S                   10000000     ucrt:api-ms-win-crt-runtime-l1-1-0.dll
 0000:fffdd000       .debug$S                   10000000     ucrt:api-ms-win-crt-runtime-l1-1-0.dll
 0000:fffdd000       .debug$S                   10000000     ucrt:api-ms-win-crt-runtime-l1-1-0.dll
 0000:fffdd000       .debug$S                   10000000     ucrt:api-ms-win-crt-runtime-l1-1-0.dll
 0000:fffdd000       .debug$S                   10000000     ucrt:api-ms-win-crt-runtime-l1-1-0.dll
 0000:fffdd000       .debug$S                   10000000     ucrt:api-ms-win-crt-runtime-l1-1-0.dll
 0000:fffdd000       .debug$S                   10000000     ucrt:api-ms-win-crt-runtime-l1-1-0.dll
 0000:fffdd000       .debug$S                   10000000     ucrt:api-ms-win-crt-runtime-l1-1-0.dll
 0000:fffdd000       .debug$S                   10000000     ucrt:api-ms-win-crt-runtime-l1-1-0.dll
 0000:fffdd000       .debug$S                   10000000     ucrt:api-ms-win-crt-runtime-l1-1-0.dll
 0000:fffdd000       .debug$S                   10000000     ucrt:api-ms-win-crt-runtime-l1-1-0.dll
 0000:fffdd000       .debug$S                   10000000     ucrt:api-ms-win-crt-runtime-l1-1-0.dll
 0000:fffdd000       .debug$S                   10000000     ucrt:api-ms-win-crt-runtime-l1-1-0.dll
 0000:fffdd000       .debug$S                   10000000     ucrt:api-ms-win-crt-runtime-l1-1-0.dll
 0000:fffdd000       .debug$S                   10000000     ucrt:api-ms-win-crt-runtime-l1-1-0.dll
 0000:fffdd000       .debug$S                   10000000     ucrt:api-ms-win-crt-runtime-l1-1-0.dll
 0000:fffdd000       .debug$S                   10000000     ucrt:api-ms-win-crt-runtime-l1-1-0.dll
 0000:fffdd000       .debug$S                   10000000     ucrt:api-ms-win-crt-runtime-l1-1-0.dll
 0000:fffdd000       .debug$S                   10000000     ucrt:api-ms-win-crt-stdio-l1-1-0.dll
 0000:fffdd000       .debug$S                   10000000     ucrt:api-ms-win-crt-stdio-l1-1-0.dll
 0000:fffdd000       .debug$S                   10000000     ucrt:api-ms-win-crt-stdio-l1-1-0.dll
 0000:fffdd000       .debug$S                   10000000     ucrt:api-ms-win-crt-stdio-l1-1-0.dll
 0000:fffdd000       .debug$S                   10000000     ucrt:api-ms-win-crt-stdio-l1-1-0.dll
 0000:fffdd000       .debug$S                   10000000     ucrt:api-ms-win-crt-stdio-l1-1-0.dll
 0000:fffdd000       .debug$S                   10000000     ucrt:api-ms-win-crt-stdio-l1-1-0.dll
 0000:fffdd000       .debug$S                   10000000     ucrt:api-ms-win-crt-string-l1-1-0.dll
 0000:fffdd000       .debug$S                   10000000     ucrt:api-ms-win-crt-string-l1-1-0.dll
 0000:fffdd000       .debug$S                   10000000     ucrt:api-ms-win-crt-string-l1-1-0.dll
 0000:fffdd000       .debug$S                   10000000     ucrt:api-ms-win-crt-string-l1-1-0.dll
 0000:fffdd000       .debug$S                   10000000     ucrt:api-ms-win-crt-string-l1-1-0.dll
 0000:fffdd000       .debug$S                   10000000     ucrt:api-ms-win-crt-time-l1-1-0.dll
 0000:fffdd000       .debug$S                   10000000     ucrt:api-ms-win-crt-time-l1-1-0.dll
 0000:fffdd000       .debug$S                   10000000     ucrt:api-ms-win-crt-utility-l1-1-0.dll
 0000:fffdd000       .debug$S                   10000000     kernel32:KERNEL32.dll
 0000:fffdd000       .debug$S                   10000000     kernel32:KERNEL32.dll
 0000:fffdd000       .debug$S                   10000000     kernel32:KERNEL32.dll
 0000:fffdd000       .debug$S                   10000000     kernel32:KERNEL32.dll
 0000:fffdd000       .debug$S                   10000000     kernel32:KERNEL32.dll
 0000:fffdd000       .debug$S                   10000000     kernel32:KERNEL32.dll
 0000:fffdd000       .debug$S                   10000000     kernel32:KERNEL32.dll
 0000:fffdd000       .debug$S                   10000000     kernel32:KERNEL32.dll
 0000:fffdd000       .debug$S                   10000000     kernel32:KERNEL32.dll
 0000:fffdd000       .debug$S                   10000000     kernel32:KERNEL32.dll
 0000:fffdd000       .debug$S                   10000000     kernel32:KERNEL32.dll
 0000:fffdd000       .debug$S                   10000000     kernel32:KERNEL32.dll
 0000:fffdd000       .debug$S                   10000000     kernel32:KERNEL32.dll
 0000:fffdd000       .debug$S                   10000000     kernel32:KERNEL32.dll
 0000:fffdd000       .debug$S                   10000000     kernel32:KERNEL32.dll
 0000:fffdd000       .debug$S                   10000000     kernel32:KERNEL32.dll
 0000:fffdd000       .debug$S                   10000000     kernel32:KERNEL32.dll
 0000:fffdd000       .debug$S                   10000000     kernel32:KERNEL32.dll
 0000:fffdd000       .debug$S                   10000000     kernel32:KERNEL32.dll
 0000:fffdd000       .debug$S                   10000000     kernel32:KERNEL32.dll
 0000:fffdd000       .debug$S                   10000000     kernel32:KERNEL32.dll
 0000:fffdd000       .debug$S                   10000000     kernel32:KERNEL32.dll
 0000:fffdd000       .debug$S                   10000000     winmm:WINMM.dll
 0000:fffdd000       .debug$S                   10000000     wsock32:WSOCK32.dll
 0000:fffdd000       .debug$S                   10000000     wsock32:WSOCK32.dll
 0000:fffdd000       .debug$S                   10000000     wsock32:WSOCK32.dll
 0000:fffdd000       .debug$S                   10000000     wsock32:WSOCK32.dll
 0000:fffdd000       .debug$S                   10000000     wsock32:WSOCK32.dll
 0000:fffdd000       .debug$S                   10000000     wsock32:WSOCK32.dll
 0000:fffdd000       .debug$S                   10000000     wsock32:WSOCK32.dll
 0000:fffdd000       .debug$S                   10000000     wsock32:WSOCK32.dll
 0000:fffdd000       .debug$S                   10000000     wsock32:WSOCK32.dll
 0000:fffdd000       .debug$S                   10000000     wsock32:WSOCK32.dll
 0000:fffdd000       .debug$S                   10000000     wsock32:WSOCK32.dll
 0000:fffdd000       .debug$S                   10000000     wsock32:WSOCK32.dll
 0000:fffdd000       .debug$S                   10000000     wsock32:WSOCK32.dll
 0001:00000000       _cleanup_item              10001000 f   hprof_loader.obj
 0001:00000000       _cleanup_item              10001000 f   hprof_monitor.obj
 0001:00000380       _check_flush               10001380 f   hprof_check.obj
 0001:000003c0       _check_heap_tags           100013c0 f   hprof_check.obj
 0001:00001fcc       $LN1580                    10002fcc     hprof_check.obj
 0001:00002004       $LN1579                    10003004     hprof_check.obj
 0001:00002104       $LN1582                    10003104     hprof_check.obj
 0001:0000213c       $LN1581                    1000313c     hprof_check.obj
 0001:0000223c       $LN1584                    1000323c     hprof_check.obj
 0001:00002244       $LN1583                    10003244     hprof_check.obj
 0001:00002250       _check_print_utf8          10003250 f   hprof_check.obj
 0001:00002330       _check_printf              10003330 f   hprof_check.obj
 0001:000023b0       _check_printf_val          100033b0 f   hprof_check.obj
 0001:000024e0       $LN23                      100034e0     hprof_check.obj
 0001:00002510       _check_raw                 10003510 f   hprof_check.obj
 0001:00002590       _check_tags                10003590 f   hprof_check.obj
 0001:0000390c       $LN755                     1000490c     hprof_check.obj
 0001:00003948       $LN754                     10004948     hprof_check.obj
 0001:00003980       _cmap_cleanup              10004980 f   hprof_check.obj
 0001:000039b0       _read_id                   100049b0 f   hprof_check.obj
 0001:000039b0       _read_u4                   100049b0 f   hprof_check.obj
 0001:000039f0       _read_u2                   100049f0 f   hprof_check.obj
 0001:00003a20       _read_u8                   10004a20 f   hprof_check.obj
 0001:00003aa0       _read_val                  10004aa0 f   hprof_check.obj
 0001:00003b74       $LN28                      10004b74     hprof_check.obj
 0001:00003b8c       $LN27                      10004b8c     hprof_check.obj
 0001:00003ba0       _system_write              10004ba0 f   hprof_check.obj
 0001:00003cd0       _utab_cleanup              10004cd0 f   hprof_check.obj
 0001:00003cf0       _all_status_remove         10004cf0 f   hprof_class.obj
 0001:000045f0       _cleanup_item              100055f0 f   hprof_class.obj
 0001:00004640       _create_entry              10005640 f   hprof_class.obj
 0001:00004720       _delete_ref_item           10005720 f   hprof_class.obj
 0001:00004760       _list_item                 10005760 f   hprof_class.obj
 0001:000047f0       _unload_walker             100057f0 f   hprof_class.obj
 0001:00004850       _cpu_loop_function@12      10005850 f   hprof_cpu.obj
 0001:00004ca0       _error_message             10005ca0 f   hprof_error.obj
 0001:00004cd0       _error_abort               10005cd0 f   hprof_error.obj
 0001:00004e50       _signal_handler            10005e50 f   hprof_error.obj
 0001:00004e70       _terminate_everything      10005e70 f   hprof_error.obj
 0001:00004ef0       _any_allocation            10005ef0 f   hprof_event.obj
 0001:00005860       _list_item                 10006860 f   hprof_frame.obj
 0001:000060e0       _cbClassFileLoadHook@40    100070e0 f   hprof_init.obj
 0001:00006450       _cbClassLoad@16            10007450 f   hprof_init.obj
 0001:00006560       _cbClassPrepare@16         10007560 f   hprof_init.obj
 0001:00006670       _cbDataDumpRequest@4       10007670 f   hprof_init.obj
 0001:000067d0       _cbExceptionCatch@28       100077d0 f   hprof_init.obj
 0001:000068a0       _cbGarbageCollectionFinish@4 100078a0 f   hprof_init.obj
 0001:00006950       _cbGarbageCollectionStart@4 10007950 f   hprof_init.obj
 0001:00006970       _cbMonitorContendedEnter@16 10007970 f   hprof_init.obj
 0001:00006a40       _cbMonitorContendedEntered@16 10007a40 f   hprof_init.obj
 0001:00006b10       _cbMonitorWait@24          10007b10 f   hprof_init.obj
 0001:00006be0       _cbMonitorWaited@20        10007be0 f   hprof_init.obj
 0001:00006cb0       _cbObjectFree@12           10007cb0 f   hprof_init.obj
 0001:00006d30       _cbThreadEnd@12            10007d30 f   hprof_init.obj
 0001:00006df0       _cbThreadStart@12          10007df0 f   hprof_init.obj
 0001:00006eb0       _cbVMDeath@8               10007eb0 f   hprof_init.obj
 0001:00007210       _cbVMInit@12               10008210 f   hprof_init.obj
 0001:00007490       _dump_all_data             10008490 f   hprof_init.obj
 0001:00007660       _gc_finish_watcher@12      10008660 f   hprof_init.obj
 0001:00007830       _get_tok                   10008830 f   hprof_init.obj
 0001:000078b0       _list_all_tables           100088b0 f   hprof_init.obj
 0001:000078e0       _lookup_library_symbol     100088e0 f   hprof_init.obj
 0001:00007990       _make_unique_filename      10008990 f   hprof_init.obj
 0001:00007af0       _my_crw_fatal_error_handler 10008af0 f   hprof_init.obj
 0001:00007b70       _option_error              10008b70 f   hprof_init.obj
 0001:00007bf0       _parse_options             10008bf0 f   hprof_init.obj
 0001:000097d0       _reset_class_load_status   1000a7d0 f   hprof_init.obj
 0001:000098a0       _setBinarySwitch           1000a8a0 f   hprof_init.obj
 0001:00009980       _set_callbacks             1000a980 f   hprof_init.obj
 0001:00009a40       _setup_event_mode          1000aa40 f   hprof_init.obj
 0001:00009b40       _dump_heap_segment_and_reset 1000ab40 f   hprof_io.obj
 0001:00009c50       _dump_instance_fields      1000ac50 f   hprof_io.obj
 0001:00009d00       _heap_element              1000ad00 f   hprof_io.obj
 0001:00009da4       $LN24                      1000ada4     hprof_io.obj
 0001:00009dd0       _heap_elements             1000add0 f   hprof_io.obj
 0001:00009f34       $LN53                      1000af34     hprof_io.obj
 0001:00009f4c       $LN52                      1000af4c     hprof_io.obj
 0001:00009f60       _heap_flush                1000af60 f   hprof_io.obj
 0001:00009fd0       _heap_printf               1000afd0 f   hprof_io.obj
 0001:0000a040       _heap_raw                  1000b040 f   hprof_io.obj
 0001:0000a0e0       _heap_tag                  1000b0e0 f   hprof_io.obj
 0001:0000a170       _heap_u2                   1000b170 f   hprof_io.obj
 0001:0000a190       _heap_u4                   1000b190 f   hprof_io.obj
 0001:0000ca80       _signature_to_name         1000da80 f   hprof_io.obj
 0001:0000cbe4       $LN39                      1000dbe4     hprof_io.obj
 0001:0000cc1c       $LN38                      1000dc1c     hprof_io.obj
 0001:0000cc50       _system_error              1000dc50 f   hprof_io.obj
 0001:0000cd60       _system_write              1000dd60 f   hprof_io.obj
 0001:0000cde0       _type_from_signature       1000dde0 f   hprof_io.obj
 0001:0000cea4       $LN18                      1000dea4     hprof_io.obj
 0001:0000cecc       $LN17                      1000decc     hprof_io.obj
 0001:0000cef0       _write_header              1000def0 f   hprof_io.obj
 0001:0000cf50       _write_name_first          1000df50 f   hprof_io.obj
 0001:0000cfd0       _write_printf              1000dfd0 f   hprof_io.obj
 0001:0000d040       _write_raw                 1000e040 f   hprof_io.obj
 0001:0000d0e0       _write_raw_from_file       1000e0e0 f   hprof_io.obj
 0001:0000d190       _write_thread_serial_number 1000e190 f   hprof_io.obj
 0001:0000d320       _listener_loop_function@12 1000e320 f   hprof_listener.obj
 0001:0000d71c       $LN58                      1000e71c     hprof_listener.obj
 0001:0000d7e0       _recv_id                   1000e7e0 f   hprof_listener.obj
 0001:0000d830       _recv_u2                   1000e830 f   hprof_listener.obj
 0001:0000d8a0       _recv_u4                   1000e8a0 f   hprof_listener.obj
 0001:0000d900       _delete_ref_item           1000e900 f   hprof_loader.obj
 0001:0000d930       _list_item                 1000e930 f   hprof_loader.obj
 0001:0000db50       _search_item               1000eb50 f   hprof_loader.obj
 0001:0000e350       _clear_item                1000f350 f   hprof_monitor.obj
 0001:0000e370       _collect_iterator          1000f370 f   hprof_monitor.obj
 0001:0000e3a0       _find_or_create_entry      1000f3a0 f   hprof_monitor.obj
 0001:0000e410       _list_item                 1000f410 f   hprof_monitor.obj
 0001:0000e9a0       _qsort_compare             1000f9a0 f   hprof_monitor.obj
 0001:0000ea10       _clear_references          1000fa10 f   hprof_object.obj
 0001:0000ea20       _dump_class_references     1000fa20 f   hprof_object.obj
 0001:0000ea40       _dump_instance_references  1000fa40 f   hprof_object.obj
 0001:0000ea60       _list_item                 1000fa60 f   hprof_object.obj
 0001:0000ede0       _dump_class_and_supers     1000fde0 f   hprof_reference.obj
 0001:0000f1e0       $LN51                      100101e0     hprof_reference.obj
 0001:0000f200       _dump_field                10010200 f   hprof_reference.obj
 0001:0000f340       _dump_fields               10010340 f   hprof_reference.obj
 0001:0000f3b0       _dump_instance             100103b0 f   hprof_reference.obj
 0001:0000f830       _dump_ref_list             10010830 f   hprof_reference.obj
 0001:0000f8a0       _fill_in_field_value       100108a0 f   hprof_reference.obj
 0001:0000f9a0       _get_prim_size             100109a0 f   hprof_reference.obj
 0001:0000f9d4       $LN15                      100109d4     hprof_reference.obj
 0001:0000f9e8       $LN14                      100109e8     hprof_reference.obj
 0001:0000fc30       _cbPrimArrayData@36        10010c30 f   hprof_site.obj
 0001:0000fc80       _cbPrimFieldData@36        10010c80 f   hprof_site.obj
 0001:0000fcf0       _cbReference@48            10010cf0 f   hprof_site.obj
 0001:000100bc       $LN51                      100110bc     hprof_site.obj
 0001:000100e0       $LN50                      100110e0     hprof_site.obj
 0001:000100fc       $LN52                      100110fc     hprof_site.obj
 0001:00010120       _collect_iterator          10011120 f   hprof_site.obj
 0001:00010150       _get_pkey                  10011150 f   hprof_site.obj
 0001:00010180       _list_item                 10011180 f   hprof_site.obj
 0001:00010220       _localReference            10011220 f   hprof_site.obj
 0001:00010390       _make_new_tag              10011390 f   hprof_site.obj
 0001:00010430       _mark_unchanged_iterator   10011430 f   hprof_site.obj
 0001:00010440       _qsort_compare_allocated_bytes 10011440 f   hprof_site.obj
 0001:00010480       _qsort_compare_live_bytes  10011480 f   hprof_site.obj
 0001:000104c0       _setup_tag_on_root         100114c0 f   hprof_site.obj
 0001:00010cd0       _list_item                 10011cd0 f   hprof_string.obj
 0001:00010e20       _find_entry                10011e20 f   hprof_table.obj
 0001:00010f60       _hashcode                  10011f60 f   hprof_table.obj
 0001:000110a0       _resize                    100120a0 f   hprof_table.obj
 0001:00011290       _setup_new_entry           10012290 f   hprof_table.obj
 0001:00011d10       _clean_in_heap_dump        10012d10 f   hprof_tls.obj
 0001:00011d20       _clean_info                10012d20 f   hprof_tls.obj
 0001:00011d70       _cleanup_item              10012d70 f   hprof_tls.obj
 0001:00011dc0       _delete_ref_item           10012dc0 f   hprof_tls.obj
 0001:00011de0       _dump_monitor_state        10012de0 f   hprof_tls.obj
 0001:00012050       _dump_thread_state         10013050 f   hprof_tls.obj
 0001:000120c0       _garbage_collect_item      100130c0 f   hprof_tls.obj
 0001:00012120       _get_thread_list           10013120 f   hprof_tls.obj
 0001:00012190       _insure_method_on_stack    10013190 f   hprof_tls.obj
 0001:00012350       _list_item                 10013350 f   hprof_tls.obj
 0001:00012380       _pop_method                10013380 f   hprof_tls.obj
 0001:00012530       _sample_setter             10013530 f   hprof_tls.obj
 0001:00012560       _search_item               10013560 f   hprof_tls.obj
 0001:000125b0       _setup_trace_buffers       100135b0 f   hprof_tls.obj
 0001:00012610       _sum_sample_status_item    10013610 f   hprof_tls.obj
 0001:00013390       _clear_cost                10014390 f   hprof_trace.obj
 0001:000133c0       _collect_iterator          100143c0 f   hprof_trace.obj
 0001:000133f0       _fill_frame_buffer         100143f0 f   hprof_trace.obj
 0001:000134b0       _find_or_create            100144b0 f   hprof_trace.obj
 0001:00013570       _list_item                 10014570 f   hprof_trace.obj
 0001:00013600       _output_list               10014600 f   hprof_trace.obj
 0001:000138f0       _output_trace              100148f0 f   hprof_trace.obj
 0001:00013b60       _qsort_compare_cost        10014b60 f   hprof_trace.obj
 0001:00013ba0       _qsort_compare_num_hits    10014ba0 f   hprof_trace.obj
 0001:00014630       _Tracker_nativeNewArray@16 10015630 f   hprof_tracker.obj
 0001:00014710       _Tracker_nativeObjectInit@16 10015710 f   hprof_tracker.obj
 0001:000147f0       _Tracker_nativeCallSite@20 100157f0 f   hprof_tracker.obj
 0001:000148e0       _Tracker_nativeReturnSite@20 100158e0 f   hprof_tracker.obj
 0001:000149d0       _set_engaged               100159d0 f   hprof_tracker.obj
 0001:00014d30       _add_class_fields          10015d30 f   hprof_util.obj
 0001:000152e4       $LN123                     100162e4     hprof_util.obj
 0001:00015308       $LN122                     10016308     hprof_util.obj
 0001:00015324       $LN125                     10016324     hprof_util.obj
 0001:00015338       $LN124                     10016338     hprof_util.obj
 0001:00016750       _get_cnum                  10017750 f   hprof_util.obj
 0001:000169e0       _jvmtiMajorVersion         100179e0 f   hprof_util.obj
 0001:00016a30       _jvmtiMinorVersion         10017a30 f   hprof_util.obj
 0001:00016b78       $LN10                      10017b78     hprof_util.obj
 0001:00016c18       $LN15                      10017c18     hprof_util.obj
 0001:00016c3c       $LN14                      10017c3c     hprof_util.obj
 0001:0001703c       $LN16                      1001803c     hprof_util.obj
 0001:00017050       $LN15                      10018050     hprof_util.obj
 0001:00017080       $$000000                   10018080     MSVCRT:lldiv.obj
 0001:000170a1       L1                         100180a1     MSVCRT:lldiv.obj
 0001:000170bd       L2                         100180bd     MSVCRT:lldiv.obj
 0001:000170d9       L3                         100180d9     MSVCRT:lldiv.obj
 0001:000170e7       L5                         100180e7     MSVCRT:lldiv.obj
 0001:00017115       L6                         10018115     MSVCRT:lldiv.obj
 0001:00017116       L7                         10018116     MSVCRT:lldiv.obj
 0001:0001711a       L4                         1001811a     MSVCRT:lldiv.obj
 0001:00017124       L8                         10018124     MSVCRT:lldiv.obj
 0001:00017130       $$000000                   10018130     MSVCRT:llshr.obj
 0001:00017140       MORE32                     10018140     MSVCRT:llshr.obj
 0001:0001714b       RETSIGN                    1001814b     MSVCRT:llshr.obj
 0001:00017160       $$000000                   10018160     MSVCRT:ftol3.obj
 0001:0001717a       _ltod3_default             1001817a     MSVCRT:ftol3.obj
 0001:000171a1       ?dllmain_crt_dispatch@@YGHQAUHINSTANCE__@@KQAX@Z 100181a1 f   MSVCRT:dll_dllmain.obj
 0001:000171f4       ?dllmain_crt_process_attach@@YAHQAUHINSTANCE__@@QAX@Z 100181f4 f   MSVCRT:dll_dllmain.obj
 0001:000172fb       ?dllmain_crt_process_detach@@YAH_N@Z 100182fb f   MSVCRT:dll_dllmain.obj
 0001:000173ab       ?dllmain_dispatch@@YAHQAUHINSTANCE__@@KQAX@Z 100183ab f   MSVCRT:dll_dllmain.obj
 0001:000174b6       ?dllmain_raw@@YGHQAUHINSTANCE__@@KQAX@Z 100184b6 f   MSVCRT:dll_dllmain.obj
 0001:000177fa       ___get_entropy             100187fa f   MSVCRT:gs_support.obj
 0001:000178cd       ?find_pe_section@@YAPAU_IMAGE_SECTION_HEADER@@QAEI@Z 100188cd f   MSVCRT:utility.obj
 0001:00017d30       $$000000                   10018d30     MSVCRT:sehprolg4.obj
 0002:00004620       _NaN                       1001d620     MSVCRT:ftol3.obj
 0002:00004624       _onept5                    1001d624     MSVCRT:ftol3.obj
 0002:00004628       _DP2to32                   1001d628     MSVCRT:ftol3.obj
 0002:00004628       _Int32ToUInt32             1001d628     MSVCRT:ftol3.obj
 0002:0000463c       _GS_ExceptionPointers      1001d63c     MSVCRT:gs_report.obj
 0002:00004b58       __sehtable$?dllmain_crt_process_attach@@YAHQAUHINSTANCE__@@QAX@Z 1001db58     MSVCRT:dll_dllmain.obj
 0002:00004b78       __sehtable$?dllmain_crt_process_detach@@YAH_N@Z 1001db78     MSVCRT:dll_dllmain.obj
 0002:00004ba0       __sehtable$?dllmain_dispatch@@YAHQAUHINSTANCE__@@KQAX@Z 1001dba0     MSVCRT:dll_dllmain.obj
 0002:00004bc0       __sehtable$___scrt_is_nonwritable_in_current_image 1001dbc0     MSVCRT:utility.obj
 0002:00004be0       .edata                     1001dbe0     hprof.exp
 0002:00004c08       rgpv                       1001dc08     hprof.exp
 0002:00004c10       rgszName                   1001dc10     hprof.exp
 0002:00004c18       rgwOrd                     1001dc18     hprof.exp
 0002:00004c1c       szName                     1001dc1c     hprof.exp
 0002:00004c26       $N00001                    1001dc26     hprof.exp
 0002:00004c37       $N00002                    1001dc37     hprof.exp
 0002:00004ec8       .idata$6                   1001dec8     wsock32:WSOCK32.dll
 0002:00004ee2       .idata$6                   1001dee2     winmm:WINMM.dll
 0002:0000508c       .idata$6                   1001e08c     kernel32:KERNEL32.dll
 0002:000050fc       .idata$6                   1001e0fc     vcruntime:VCRUNTIME140.dll
 0002:000052f0       .idata$6                   1001e2f0     ucrt:api-ms-win-crt-runtime-l1-1-0.dll
 0002:00005312       .idata$6                   1001e312     ucrt:api-ms-win-crt-string-l1-1-0.dll
 0002:00005334       .idata$6                   1001e334     ucrt:api-ms-win-crt-stdio-l1-1-0.dll
 0002:00005354       .idata$6                   1001e354     ucrt:api-ms-win-crt-filesystem-l1-1-0.dll
 0002:0000537a       .idata$6                   1001e37a     ucrt:api-ms-win-crt-heap-l1-1-0.dll
 0002:0000539a       .idata$6                   1001e39a     ucrt:api-ms-win-crt-convert-l1-1-0.dll
 0002:000053bc       .idata$6                   1001e3bc     ucrt:api-ms-win-crt-environment-l1-1-0.dll
 0002:000053e2       .idata$6                   1001e3e2     ucrt:api-ms-win-crt-time-l1-1-0.dll
 0002:00005402       .idata$6                   1001e402     ucrt:api-ms-win-crt-utility-l1-1-0.dll
 0003:00000000       _type_size                 1001f000     hprof_check.obj
 0003:00000030       ?signatures@?1??class_prime_system_classes@@9@9 1001f030     hprof_class.obj
 0003:00000050       _p                         1001f050     hprof_error.obj
 0003:00000054       ?symbols@?O@??Agent_OnLoad@@9@9 1001f054     hprof_init.obj
 0003:0000005c       ?symbols@?P@??Agent_OnLoad@@9@9 1001f05c     hprof_init.obj
 0003:00000064       _type_size                 1001f064     hprof_io.obj
 0003:00000094       ?pid@?1??md_getpid@@9@9    1001f094     hprof_md.obj
 0003:00000098       _registry                  1001f098     hprof_tracker.obj
 0003:000000c8       _tracker_methods           1001f0c8     hprof_tracker.obj
 0003:00000138       ?empty_val@?1??read_val@@9@9 1001f138     hprof_check.obj
 0003:00000140       ?empty_key@?1??fillin_pkey@@9@9 1001f140     hprof_class.obj
 0003:00000148       ?empty_key@?1??frame_find_or_create@@9@9 1001f148     hprof_frame.obj
 0003:00000158       ?data@?1??get_gdata@@9@9   1001f158     hprof_init.obj
 0003:000003d8       ?empty_val@?1??heap_elements@@9@9 1001f3d8     hprof_io.obj
 0003:000003e0       ?empty_info@?4??loader_find_or_create@@9@9 1001f3e0     hprof_loader.obj
 0003:000003e8       ?fileTime_1_1_70@?1??md_get_timemillis@@9@9 1001f3e8     hprof_md.obj
 0003:000003f0       _nError                    1001f3f0     hprof_md.obj
 0003:000003f4       ?empty_key@?1??object_new@@9@9 1001f3f4     hprof_object.obj
 0003:00000404       ?empty_info@?2??object_new@@9@9 1001f404     hprof_object.obj
 0003:00000410       ?empty_value@?1??get_key_value@@9@9 1001f410     hprof_reference.obj
 0003:00000418       ?empty_value@?L@??dump_class_and_supers@@9@9 1001f418     hprof_reference.obj
 0003:00000420       ?empty_value@?M@??dump_instance@@9@9 1001f420     hprof_reference.obj
 0003:00000428       ?empty_info@?1??reference_obj@@9@9 1001f428     hprof_reference.obj
 0003:0000043c       ?empty_info@?1??reference_prim_field@@9@9 1001f43c     hprof_reference.obj
 0003:00000450       ?empty_info@?1??reference_prim_array@@9@9 1001f450     hprof_reference.obj
 0003:00000468       ?empty_info@?1??tls_find_or_create@@9@9 1001f468     hprof_tls.obj
 0003:000004a8       ?empty_key@?1??find_or_create@@9@9 1001f4a8     hprof_trace.obj
 0003:000004b8       ?empty_finfo@?O@??add_class_fields@@9@9 1001f4b8     hprof_util.obj
 0003:000004c8       ?__proc_attached@@3HA      1001f4c8     MSVCRT:dll_dllmain.obj
 0003:000004d0       _GS_ExceptionRecord        1001f4d0     MSVCRT:gs_report.obj
 0003:00000520       _GS_ContextRecord          1001f520     MSVCRT:gs_report.obj
 0003:00000810       ?is_initialized_as_dll@@3_NA 1001f810     MSVCRT:utility.obj
 0003:00000811       ?module_local_atexit_table_initialized@@3_NA 1001f811     MSVCRT:utility.obj
 0003:00000814       ?module_local_atexit_table@@3U_onexit_table_t@@A 1001f814     MSVCRT:utility.obj
 0003:00000820       ?module_local_at_quick_exit_table@@3U_onexit_table_t@@A 1001f820     MSVCRT:utility.obj
 0004:00000060       $R000000                   10020060     hprof.dll.res
